:10000E00000000C0F0F87C7C7C7CF8F0C0000000A2
:10001E000000FCFF1F010000000001DFFFFE0000DA
:10002E0000FEFFFF0000C0E0F8FE3F0FFFFFFE00E6
:10003E00007FFFFFFC3F1F0701000000FFFF1F00B6
:10004E0000001FFFFCC080000080E0FCFF1F0000CE
:10005E0000000001070F0F1F1F0F07030000000015
:10006E0000000080C0E0F0F8FCFC00000000000082
:10007E0000000E1F0F0701FFFFFF00000000000031
:10008E0000000000000000FFFFFF00000000000065
:10009E0000000000000000FFFFFF00000000000055
:1000AE0000008080808080FFFFFF808080800000C5
:1000BE0000000F0F0F0F0F0F0F0F0F0F0F0F00007E
:1000CE00000080E0F0F87C7C7CFCF8E08000000012
:1000DE00000000070100000000000FFFFF000000FD
:1000EE00000000000000000000C0FEFF1F00000026
:1000FE00000000000080E0F8FE3F07010000000055
:10010E000000C0F0FCBF8F83808080808080000064
:10011E0000000F0F0F0F0F0F0F0F0F0F0F0F00001D
:10012E00000000F8787C7C7C7CF8F8E08000000011
:10013E0000000000000000000000FFFFFF000000B4
:10014E000000000000F0F0F0F0FCDF8F0100000076
:10015E000000000000010101010307FFFEF800008E
:10016E00000080800000000080C0E0FFFF0F000054
:10017E0000000F0F0F1F1F0F0F0F070100000000D1
:10018E0000000000000000C0F8F8F8F800000000C1
:10019E000000000000E0FE7F0700FFFF00000000EF
:1001AE00000080F0FF3F03000000FFFF0000000092
:1001BE0000F8FFDFC1C0C0C0C0C0FFFFC0C0C0009C
:1001CE0000070707070707070707FFFF07070700CF
:1001DE00000000000000000000000F0F00000000F3
:1001EE00000000F8F8787878787878787800000051
:1001FE00000000FFFF0000000000000000000000F3
:10020E00000000FFFFF8F8F8F8F0F0E080000000C2
:10021E000000000000000000000107FFFFFC0000CE
:10022E00000000800000000080C0F0FF7F0700008B
:10023E000000000F0F1F1F0F0F070301000000002B
:10024E000000000080C0E0F0F8F878787800000038
:10025E00000080FCFF0F0301000000000000000002
:10026E000000FFFFE1F0F8787C78F8F0E080000005
:10027E000000FFFF0100000000000007FFFF00006C
:10028E0000001FFFFFC080000000C0F0FF7F0000D5
:10029E0000000000030F0F1F1F0F0F0701000000CB
:1002AE000000F8F8F8F8F8F8F8F8F8F8F8F80000A0
:1002BE0000000000000000000000E0FF7F070000CB
:1002CE000000000000000000C0FEFF0F0000000054
:1002DE0000000000000080FCFF3F01000000000055
:1002EE000000000000F8FF7F030000000000000087
:1002FE00000000000F0F0F000000000000000000C3
:10030E00000000E0F0F87C7C7C7CF8F8E000000057
:10031E000000FFFFFF000000000000FFFFFF0000D5
:10032E000000010F1FFFFCF8F0FCFE1F070000008D
:10033E000000F0FCFF0F070103071FFFFEF0000097
:10034E000000FFFFF0C080000080C0F0FF7F0000C3
:10035E0000000003070F0F1F1F0F0F070300000001
:10036E00000000E0F0F87C3C7C7CF8F0800000009F
:10037E0000E0FFFF07000000000001FFFFF8000093
:10038E000003FFFFF08080008080C0E0FFFF0000D0
:10039E0000000003070F0F0F0F0707F3FFFF00000A
:1003AE0000000080808080C0E0F0FC7F0F00000025
:1003BE000000000F0F0F0F070703010000000000E1
:1003CE0000F03C0E0E1CF80000FFE0381C07FF7F0B
:1003DE00000F1C3030380F000070381CFE0000007B
:1003EE0000000000FF000000003838383F383800A9
:1003FE0000181C0E0EFCF000000000C0F03F0700BD
:10040E0000383E3B38383800000C0C0E0EFCF00065
:10041E0000001C1C1C3FE10000303030301C0F006F
:10042E00000000E03CFC0000C0F88F8180FF80805F
:10043E0001010101013F010100FCFC0C0C0C0C0040
:10044E00000F0F0C0C3CF00000303030381C070051
:10045E0000C0F01C0C0C0C0000FF1C0C0E0CF80065
:10046E0000071E3030380F00000C0C0C0CCCFC00BA
:10047E0000000080F80F00000000381F010000008F
:10048E0000F09C0E0E0CF80000C1771E1C7FE300DE
:10049E00001F383030381F0000F01C0E0E1CF0000C
:1004AE00001F38303018FF0000303038180E0300AF
:1004BE0000000000000000000000F03C0C0C0C00DE
:1004CE000000F03C0C0C0CFC03030303FC00000CBE
:1004DE000CFF0C0C0C00000C0CFF0C0C0C000F3065
:1004EE003030300F000000003F0000000000000020
:1004FE003F00000000C03030C000C030303030C08F
:10050E00030C0C0300FF00000000030000000000BD
:10051E000F303030300F00F00000000000F000000F
:10052E003FC000C03F000000000F300F0000000071
:10053E0000003C3CF00C030303030303030303031B
:10054E00030303030303030303030303030303036D
:10055E00030303030303030303030303030303035D
:10056E000303030303030303030CF00F30C0C0C0E7
:10057E00C0C0C0C0C0C0C0C0C0C0C0C0C0C0C0C06D
:10058E00C0C0C0C0C0C0C0C0C0C0C0C0C0C0C0C05D
:10059E00C0C0C0C0C0C0C0C0C0C0C0C0C0C0C0C04D
:1005AE00300F000CF00C0C0C300000000F3030300F
:1005BE000C0000FC0C0C0CF0000000FF0303030009
:1005CE000000C0F0FCFCFCFCFCFCFCFCFCFCFCFC9D
:1005DE00FCFCFCFCFCFCFCFCFCFCFCFCFCFCFCFC4D
:1005EE00FCFCFCFCFCFCFCFCFCFCF0C0FFFFFFFF79
:1005FE00FFFFFFFF00FFFFF3F3F3F3F3F3F3F3F368
:10060E00FFFFFFFFF30FFFFF03F3F3F3F3F303FF1C
:10061E00FFFFFFFFFFFFFFFFFFFFFFFF03FF00FCDA
:10062E00F3FF003C3C3C3C3C00FFFFFFFCC3FF3FA4
:10063E00FFFF003C3C3C3C3C00FFFFFFFFFFFFFF89
:10064E00FFFFFFFFFFFCFFFF00FFFFFF00CFCFCF3D
:10065E00CFCF00FFFFFFCFCF03FCFF03F3F303F376
:10066E0003F3F303FFFFFFFFFFFFFFFFFFFFFFFF9C
:10067E00FFFF00FFFFCFCFCFCFCFCFCFCFCFFFFF2B
:10068E00FFFFC0FFCFC0CFCFC0CFC0CFCFC0CFFFF7
:10069E00FFFFFFFF030F3F3F3F3F3F3F3F3F3F3FC8
:1006AE003F3F3F3F3F3F3F3F3F3F3F3F3F3F3F3F4C
:1006BE003F3F3F3F3F3F3F3F3F3F3F3F0F03C0F076
:1006CE00FCFCFCFCFCFCFCFCFCFCFCFCFCFCFCFC5C
:1006DE00FCFCFCFCFCFCFCFCFCFCFCFCFCFCFCFC4C
:1006EE00FCFCFCFCFCFCF0C0FFFFFFFFFFFFFFFF6C
:1006FE0000FFFFFFFFFF3F3F3F3F3FFFFFFF3F3F3B
:10070E003F003F3FFF3F3F003F3F3FFFFFFFFFFFE9
:10071E00FFFFFFFFFFFFFFFCFCFC00FCFC00FFFFE8
:10072E0000FFFFFF00FFFFFFFFFF3F00CFCFFFFFE8
:10073E00CF00FFFF00FFFFFFFFFFFFFFFFFFFFFFE9
:10074E00FFFFFFFF00FFFF00FFFF00FFFFFF00FFA7
:10075E00FFFFFCCC3FC0FFFF3FCFF0FFF0FFF0CF1D
:10076E0000FFFFFFFFFFFFFFFFFFFF3FCFF0FFCFB9
:10077E003FC0FFFFC0F3F3F3C0FFFFFF3FC3FFFF18
:10078E00F30FFFFFF30FFFFFF30FFFFFFFFFFFFF5F
:10079E00030F3F3F3F3F3F3F3F3F3F3F3F3F3F3FC7
:1007AE003F3F3F3F3F3F3F3F3F3F3F3F3F3F3F3F4B
:1007BE003F3F3F3F3F3F3F3F0F03C0300C0C0C0C01
:1007CE000C0C0C0C0C0C0C0C0C0C0C0C0C0C0C0C5B
:1007DE000C0C0C0C0C0C0C0C0C0C0C0C0C0C0C0C4B
:1007EE000C0C30C0FF0000000000000000033C00B5
:1007FE0000000000300F0000000000C0030C000CD1
:10080E000C0CCC0C0C0C0CFC0000000000FFFF00CC
:10081E000000000000000303030303FF03030303B0
:10082E000300000000FF000C0C0C0CCCFF0C0C0C99
:10083E0000FF0000000000FFFF00000000000303A7
:10084E0003030303F30FF30303030303030000FF88
:10085E0000C0300C0300FF00000000FF000000008D
:10086E0000FFFF0000000000C0C030300C0300008D
:10087E0000030C3030C0C00000FF00000000030C6D
:10088E0003000030C03F0000000000FF030C3030BA
:10089E00303030303030303030303030303030304A
:1008AE00303030303030303030303030303030303A
:1008BE00303030300C0300F0FCFCFFFFFFFFFFFF79
:1008CE00FFFFFFFFFFFFFFFFFFFFFFFFFFFFFFFF2A
:1008DE00FFFFFCFCF000FFFFFFFFFFFFFFFFFFFF2E
:1008EE00FFFFFFFFFFFFFFFFFFFFFFFFFFFFFFFF0A
:1008FE00FFFFFFFFFFFFFFFFFFFFFF3F3F3F3F3FBA
:10090E003FFFFF3F3F3F3F3FFF3F3F3F3F3F3FFFE9
:10091E00FFFFFFFFFFFFFFFFFFFFFFFF00FFFFFFD8
:10092E00FF00FFFFFF00FFFFFFFF00FFFFFFFFFCC9
:10093E0003FFFFFFFFFFFFFFFFFFFFFF00FCFCFCBD
:10094E00FCFFFFFFFF00FFFFFFFF00FFFFFFFFFFAA
:10095E0000FFFFFFFFFFFFFFFFFFFFF3F0F3FFFFBF
:10096E00FFFFFFF3F3F0F3F3FFF3F0F3F3F3F3FC16
:10097E00FFFFFFFFFFFFFFFFFFFFFFFFFFFFFFFF79
:10098E00FFFFFFFFFFFFFFFFFFFFFFFFFFFFFFFF69
:10099E00FFFFFFFFFFFF000F3F3FFFFFFFFFFFFFC8
:1009AE00FFFFFFFFFFFFFFFFFFFFFFFFFFFFFFFF49
:1009BE00FFFF3F3F0F0000F0FCFCFFFFFFFFFFFFBC
:1009CE00FFFFFFFFFFFFFFFFFFFFFFFFFFFFFFFF29
:1009DE00FFFFFCFCF000FFFFFFFFFFFFFFFFFFFF2D
:1009EE00FFFFFFFFFFFFFFFFFFFFFFFFFFFFFFFF09
:1009FE00FFFFFFFFFFFFFFFFFFCF3FFFFF03F3F3FD
:100A0E00F3F303FFFFFFFFFF3F3F3F3F330F3F3F38
:100A1E003F3F3FFFFFFFFFFFF3CFFFFFFF003C3CD9
:100A2E003C3C00FFFFFFFFFF00F3F3003333333393
:100A3E0000F3F3FFFFFFFFFFFF0FF0FF03F303F3DE
:100A4E00F303F303FFFFFFFF00FFF3C333F3F333AF
:100A5E00C3F3FFFFFFFFFFFFF0FFFFCFC0CFC0CFFD
:100A6E00CFC0CFC0CFFFCFF0FFCFCFF3F3FCFCF35F
:100A7E00F3CFCFFFFFFFFFFFFFFFFFFFFFFFFFFFE4
:100A8E00FFFFFFFFFFFFFFFFFFFFFFFFFFFFFFFF68
:100A9E00FFFFFFFFFFFF000F3F3FFFFFFFFFFFFFC7
:100AAE00FFFFFFFFFFFFFFFFFFFFFFFFFFFFFFFF48
:100ABE00FFFF3F3F0F0000F0FCFCFFFFFFFFFFFFBB
:100ACE00FFFFFFFFFFFFFFFFFFFFFFFFFFFFFFFF28
:100ADE00FFFFFCFCF000FFFFFFFFFFFFFFFFFFFF2C
:100AEE00FFFFFFFFFFFFFFFFFFFFFFFFFFFFFFFF08
:100AFE00FFFFFFFFFFFFFFFFFFFFFF03FFFF3F03B0
:100B0E003F3F3F033F3FFFFFFFFFFFFFFFFF03FF9F
:100B1E00F3CFFFFFFFFFFFFFFFFC3C003CFF033066
:100B2E003333333003FFFC3C3C3C3C3CFCFC00FCD0
:100B3E00FCFCFCFFFFFFFFFFFFF3FC00FF3C30332C
:100B4E0033033333303FFFFFFF00FFFFFFFFF00F94
:100B5E00FFFF3FFFFFFFFFFFFFFFFFC0FFCFCFF302
:100B6E00FCFFFCF3CFCFF3F3F3F0FCFCFCFFFFFF35
:100B7E00FCF3C0FFFFFFFFFFFFFFFFFFFFFFFFFFC5
:100B8E00FFFFFFFFFFFFFFFFFFFFFFFFFFFFFFFF67
:100B9E00FFFFFFFFFFFF000F3F3FFFFFFFFFFFFFC6
:100BAE00FFFFFFFFFFFFFFFFFFFFFFFFFFFFFFFF47
:100BBE00FFFF3F3F0F0000F0FCFCFFFFFFFFFFFFBA
:100BCE00FFFFFFFFFFFFFFFFFFFFFFFFFFFFFFFF27
:100BDE00FFFFFCFCF000FFFFFFFFFFFFFFFFFFFF2B
:100BEE00FFFFFFFFFFFFFFFFFFFFFFFFFFFFFFFF07
:100BFE00FFFFFFFFFFFFFFFFFFCF3FFFFF0FCFCF37
:100C0E00CFCF0FFFFFFFFF0FFFFFFFFF03FFFFFF22
:100C1E00FF0FFFFFFFFFFFFF3F3F3CFFFF00CC0C2E
:100C2E00CCCCC03FFFFFFFC0CFCFCFCF00CFCFCFB9
:100C3E00CFC0FFFFFFFFFFFFFFFF00FFFF003FCF13
:100C4E00FCF3CC3FFFFF03FFFFFFFFFF00FFFFFFA3
:100C5E00FFFF03FFFFFFFFFFCFF3FCF3CFCCCFCFA0
:100C6E00CFCFCFCCCFFFF0F3F3F3F3F3F0F3F3F3F7
:100C7E00F3F3C0FFFFFFFFFFFFFFFFFFFFFFFFFFCD
:100C8E00FFFFFFFFFFFFFFFFFFFFFFFFFFFFFFFF66
:100C9E00FFFFFFFFFFFF000F3F3FFFFFFFFFFFFFC5
:100CAE00FFFFFFFFFFFFFFFFFFFFFFFFFFFFFFFF46
:100CBE00FFFF3F3F0F00000000000000000000009B
:100CCE000000C0C0C0000000000000C0C0F0F0FC7A
:100CDE00FCFFFFFFFFFFFFFCC0FCFFFFFFFFFFFF5E
:100CEE00FFFFFFFFFFFFFFFFFF033FFFFFFFFFFFC2
:100CFE00FFFFFFFFFFFFFFFFFFFF000000000303EA
:100D0E000F0F3F3FFFFFFFFFFFFF3F000000000000
:100D1E000000000000000003030300000000C0C03C
:100D2E00C0000000000000000000000000FCFFFFFB
:100D3E00FFFFFFFFFCFCF0F0C0C000000000FFFF53
:100D4E00FFFFFFFFFFFFFFFFFFFFFFFFFFFCC0FFE7
:100D5E00FFFFFFFFFFFFFFFFFFFFFFFFFFFF3F0351
:100D6E003FFFFFFFFFFFFF3F3F0F0F03030000009A
:100D7E00000000030303000000000000000000005C
:100D8E000000000000000000000000000000C0C0D5
:100D9E00C0000000000000C0C0F0F0FCFCFF3F3FB0
:100DAE000FFFFFFCC0FCFFFF3F0F0F03030000000F
:100DBE000000FFFFFF033FFFFFFCF0F0C0C000008C
:100DCE00000000FFFFFF0000000003030F0F3F3F76
:100DDE00FFFCFCF0FFFF3F000000000000000000E1
:100DEE00000000030303000000000030CCFCFCCC2C
:100DFE003000000030CCFCFCFCFCFCFCFCFCCC30DD
:100E0E000000C0C0C0000000000000000000000094
:100E1E0000FCFFFF0F3F3FFFFCFCF0F0C0C00000E6
:100E2E000000FFFFFF000000000003030F0F3FFF55
:100E3E00FFFCC0FFFFFF0000000000C0C0F0F0FC90
:100E4E00FFFF3F033FFFFFF0FCFCFF3F3F0F0F0391
:100E5E000300000000000003030300000000000078
:100E6E0000000000000000F0FCFCFFFFFFFFFFFF92
:100E7E00FFFFFFFFFFFFFFFFFFFFFFFFFFFFFCFC7A
:100E8E00F000FFFFFFFFFFFFFFFFFFFFFFFFFFFF72
:100E9E00FFFFFFFFFFFFFFFFFFFFFFFFFFFFFFFF54
:100EAE00FFFFFFFF00FFFF3FCFF3FCFFFF00FCFC47
:100EBE00FCFCF30FFFFFFFFFFFFFFFFFFFFFFFFF36
:100ECE0000F3CC3FFFFFFFFFFF00CFCFCFCFF3FCF0
:100EDE00FFFFFFFFFFFFFFFFFFFFFFFFC0FFFFFF53
:100EEE00FCF3CFFFFFC0FFFFFFFFFFFFFFFFFFFF82
:100EFE00FFFFFFFFFFFFFFFFFFFFFFFFFFFFFFFFF4
:100F0E00FFFFFFFFFFFFFFFFFFFFFFFFFFFF000FD2
:100F1E003F3FFFFFFFFFFFFFFFFFFFFFFFFFFFFF53
:100F2E00FFFFFFFFFFFF3F3F0F0000F0FCFCFFFF46
:100F3E00FFFFFFFFFFFFFFFFFFFFFFFFFFFFFFFFB3
:100F4E00FFFFFCFCF000FFFFFFFFFFFFFFFFFFFFB7
:100F5E00FFFFFFFFFFFFFFFFFFFFFFFFFFFFFFFF93
:100F6E00FFFFFFFFFFFFFFFF00FFFF3FCFF3FCFF81
:100F7E00FFFCFCFC00FCFCFCFFFFFFFFFFFFFFFF84
:100F8E00FFFFFFFF00F3CC3FFFFFFFFFFFFFFFFF61
:100F9E0000FFFFFFFFFFFFFFFFFFFFFFFFFFFFFF52
:100FAE00C0FFFFFFFCF3CFFFFFCFCFCFC0CFCFCF20
:100FBE00FFFFFFFFFFFFFFFFFFFFFFFFFFFFFFFF33
:100FCE00FFFFFFFFFFFFFFFFFFFFFFFFFFFFFFFF23
:100FDE00FFFF000F3F3FFFFFFFFFFFFFFFFFFFFF82
:100FEE00FFFFFFFFFFFFFFFFFFFF3F3F0F0000F080
:100FFE00FCFCFFFFFFFFFFFFFFFFFFFFFFFFFFFFF9
:10100E00FFFFFFFFFFFFFCFCF000FFFFFFFFFFFFF6
:10101E00FFFFFFFFFFFFFFFFFFFFFFFFFFFFFFFFD2
:10102E00FFFFFFFFFFFFFFFFFFFFFFFF00FFFF3F81
:10103E00CFF3FCFFFF00FCFCFCFCC33FFFFFFFFFF8
:10104E00FFFFFFFFFFFFFFFF00F3CC3FFFFFFFFFA0
:10105E00FF00FFFFFFFFFF00FFFFFFFFFFFFFFFF90
:10106E00FFFFFFFFC0FFFFFFFCF3CFFFFFC0CFCF9F
:10107E00CFCFF0FFFFFFFFFFFFFFFFFFFFFFFFFFE1
:10108E00FFFFFFFFFFFFFFFFFFFFFFFFFFFFFFFF62
:10109E00FFFFFFFFFFFF000F3F3FFFFFFFFFFFFFC1
:1010AE00FFFFFFFFFFFFFFFFFFFFFFFFFFFF3F3FC2
:1010BE000F0000F0FCFCFFFFFFFFFFFFFFFFFFFF35
:1010CE00FFFFFFFFFFFFFFFFFFFFFCFCF000FFFF36
:1010DE00FFFFFFFFFFFFFFFFFFFFFFFFFFFFFFFF12
:1010EE00FFFFFFFFFFFFFFFFFFFFFFFFFFFFFFFF02
:1010FE00CFCF03030000CFCFCFCFCFCFCFCF3FFF88
:10110E00FFFFFFFFFFFFFFFFFFFFFFFFFFFFFFFFE1
:10111E00FCFCFFFFFFFFFFFFFFFFFF00FFFFFFFFD6
:10112E00FFFFFFFFFFFFFFFFF3F3F3F3F3F3F3F321
:10113E00F3F3F3F3F3F3FCFFFFFFFFFFFFFFFFFFFC
:10114E00FFFFFFFFFFFFFFFFFFFFFFFFFFFFFFFFA1
:10115E00FFFFFFFFFFFFFFFFFFFF000F3F3FFFFF00
:10116E00FFFFFFFFFFFFFFFFFFFFFFFFFFFFFFFF81
:10117E00FFFF3F3F0F0000F00C0C030303030303BC
:10118E0003030303030303030303030303030C0C0F
:10119E00F000FF0000000000000000000000000052
:1011AE0000000000000000000000000000FFFF0033
:1011BE0000000000FF0000C0300C030000FF03031E
:1011CE0003030CF00000000000FFFF000000000011
:1011DE00FF0C33C00000000000FF303030300C0335
:1011EE000000000000FFFF00000000003F000000B4
:1011FE00030C3000003F0000000000000000000063
:10120E0000FFFF00000000000000000000000000D2
:10121E0000000000000000000000000000FF000FB2
:10122E003030C0C0C0C0C0C0C0C0C0C0C0C0C0C0D0
:10123E00C0C0C0C0C0C030300F0000F00C0C0303A3
:10124E000303030303030303030303030303030360
:10125E0003030C0CF000FF00000000000000000073
:10126E000000000000000000000000000000000070
:10127E0000FFFF0000000000FF0000C0300C030064
:10128E0000030303FF0303030000000000FFFF0041
:10129E0000000000FF0C33C0000000000000000042
:1012AE00FF0000000000000000FFFF000000000033
:1012BE003F000000030C3000003030303F30303043
:1012CE000000000000FFFF00000000000000000012
:1012DE000000000000000000000000000000000000
:1012EE0000FF000F3030C0C0C0C0C0C0C0C0C0C002
:1012FE00C0C0C0C0C0C0C0C0C0C030300F0000F001
:10130E000C0C03030303030303030303030303038D
:10131E000303030303030C0CF000FF0000000000A6
:10132E0000000000000000000000000000000000AF
:10133E000000000000FFFF0000000000FF0000C0E2
:10134E00300C030000FF030303033CF00000000019
:10135E0000FFFF0000000000FF0C33C00000000083
:10136E0000FF0000000000FF0000000000FFFF0073
:10137E00000000003F000000030C3000003F303042
:10138E00303C0F000000000000FFFF0000000000D6
:10139E00000000000000000000000000000000003F
:1013AE000000000000FF000F3030C0C0C0C0C0C041
:1013BE00C0C0C0C0C0C0C0C0C0C0C0C0C0C030303F
:1013CE000F0000F0FCFCFFFFFFFFFFFFFFFFFFFF22
:1013DE00FFFFFFFFFFFFFFFFFFFFFCFCF000FFFF23
:1013EE00FFFFFFFFFFFFFFFFFFFFFFFFFFFFFFFFFF
:1013FE00FFFFFFFFFFFFFFFFFFFFFFFFFFF30303F3
:10140E00FF0303F3FFFFFF3FC33FFFFFFFF3C333B2
:10141E00FF33C3F3FFFFFFFFFFFF00F00FF000FFEE
:10142E00FFFF3F003F003FFFFFFFFF3CC33CFFFFBE
:10143E00FFFFFFFFFFCFC0FFC0FFC0CFFFCFC0CF6A
:10144E00FFCFC0CFFFCFC3CCFFCCC3CFFFFFFFFF7B
:10145E00FFFFFFFFFFFFFFFFFFFFFFFFFFFFFFFF8E
:10146E00FFFFFFFFFFFFFFFFFFFF000F3F3FFFFFED
:10147E00FFFFFFFFFFFFFFFFFFFFFFFFFFFFFFFF6E
:10148E00FFFF3F3F0F0000F0FCFCFFFFFFFFFFFFE1
:10149E00FFFFFFFFFFFFFFFFFFFFFFFFFFFFFCFC54
:1014AE00F000FFFFFFFFFFFFFFFFFFFFFFFFFFFF4C
:1014BE00FFFFFFFFFFFFFFFFFFFFFFFFFFFFFFFF2E
:1014CE00FFF30303FF0303F3FFFFF3F303F3F3FF52
:1014DE00FFF30303FFF303F3FFFFFFFFFFFF00F034
:1014EE000FF000FFFFFFFFFF00FFFFFFFFFF00FFFA
:1014FE00C03F00FFFFFFFFFFFFCFC0FFC0FFC0CF09
:10150E00FFFFCFCFC0CFCFFFFFCFC0CFFFF0C0FFC9
:10151E00FFFFFFFFFFFFFFFFFFFFFFFFFFFFFFFFCD
:10152E00FFFFFFFFFFFFFFFFFFFFFFFFFFFF000FAC
:10153E003F3FFFFFFFFFFFFFFFFFFFFFFFFFFFFF2D
:10154E00FFFFFFFFFFFF3F3F0F0000F0FCFCFFFF20
:10155E00FFFFFFFFFFFFFFFFFFFFFFFFFFFFFFFF8D
:10156E00FFFFFCFCF000FFFFFFFFFFFFFFFFFFFF91
:10157E00FFFFFFFFFFFFFFFFFFFFFFFFFFFFFFFF6D
:10158E00FFFFFFFFFFFFFFFFCFCF03030000CFCF13
:10159E00CFCFCFCFCFCF3FFFFFFFFFFFFFFFFFFF2D
:1015AE00FFFFFFFFFFFFFFFFFCFCFFFFFFFFFFFF43
:1015BE00FFFFFF00FFFFFFFFFFFFFFFFFFFFFFFF2C
:1015CE00F3F3F3F3F3F3F3F3F3F3F3F3F3F3FCFFC8
:1015DE00FFFFFFFFFFFFFFFFFFFFFFFFFFFFFFFF0D
:1015EE00FFFFFFFFFFFFFFFFFFFFFFFFFFFFFFFFFD
:1015FE00FFFF000F3F3FFFFFFFFFFFFFFFFFFFFF5C
:10160E00FFFFFFFFFFFFFFFFFFFF3F3F0F0000F059
:10161E000C0C03030303030303030303030303037A
:10162E000303030303030C0CF000FF000000000093
:10163E00000000000000000000000000000000009C
:10164E000000000000FFFF00000CFCFC00FCFC0C86
:10165E00000000C03CC00000000C3CCC00CC3C0C98
:10166E0000FFFF000000FF0FF00FFF000000C0FFA3
:10167E00C0FFC000000000C33CC3000000FFFF001D
:10168E0000303F003F003F3000303F3000303F30F1
:10169E0000303C3300333C3000FFFF000000000000
:1016AE00000000000000000000000000000000002C
:1016BE000000000000FF000F3030C0C0C0C0C0C02E
:1016CE00C0C0C0C0C0C0C0C0C0C0C0C0C0C030302C
:1016DE000F0000F00C0C03030303030303030303C7
:1016EE00030303030303030303030C0CF000FF00C7
:1016FE0000000000000000000000000000000000DC
:10170E00000000000000000000FFFF00000CFCFCC9
:10171E0000FCFC0C00000C0CFC0C0C00000CFCFC87
:10172E00000CFC0C00FFFF000000FF0FF00FFF008D
:10173E0000000000FF0000000000FF003FC0FF009F
:10174E0000FFFF0000303F003F003F300000303010
:10175E003F30300000303F30000F3F0000FFFF00F1
:10176E00000000000000000000000000000000006B
:10177E00000000000000000000FF000F3030C0C06D
:10178E00C0C0C0C0C0C0C0C0C0C0C0C0C0C0C0C04B
:10179E00C0C030300F0000F00000000000FC000060
:1017AE00000000000000C03C0030F030303000007F
:1017BE00FC0030303030F0300C0C0C0C00000030DF
:1017CE00C000FC00C0300000FC00000000FF303004
:1017DE00303000FFC0300C030000300CFF0000F072
:1017EE000F0CFC00FF00FF0000303C33F030300CDB
:1017FE00C300000000C3330FFF0F33C3C03CC3034D
:10180E00FF0300FF0000C00000FF0000000000000A
:10181E000000FF000C030CF00F003F00FF000C0C4B
:10182E00CF0F0CFC0C0CCC0F3C00000CCCFF0C0CA6
:10183E00FC0000003FC03F00003F0C030000000F03
:10184E00303030303F0000003F00300C030000000D
:10185E0030303F000C030030303F000000030C001E
:10186E000030300C0F030C3000300C030C30C0C0B5
:10187E00C0303000F030303030F00000000000C0DA
:10188E003C0000003CC00000000030303030F03032
:10189E000C0C0C0C00000030C000FC00C03000002E
:1018AE00FC0000003030FF303000FF00000000FF71
:1018BE000000C030CCC3C0C0C0C0C0C30C30C0001C
:1018CE0000303C33F030300CC300000000C3330F47
:1018DE00FF0F33C3C03CC303FF03C03CFF030C0028
:1018EE0003C30303C3030000000000C03F00000059
:1018FE0000FF000000000C0CCF0F0CFC0C0CCC0FEA
:10190E003C00000CCCFF0C0CFC0000003FC03F0064
:10191E0000003F0000300C03000000033C00300CC0
:10192E00030000000030300F000000000C030030F8
:10193E00303F000000030C000030300C0F030C3061
:10194E0000300C030C3000C03CF000FC00F000FC3A
:10195E0000000000000000C03C0000003CC0000081
:10196E00000030303030F0300C0C0C0C0000003029
:10197E00C000FC00C0300000FC00000003C03CC3EF
:10198E00C3C3C3C30CF303FF0300C030CCC3C0C03A
:10199E00C0C0C0C30C30C00000303C33F030300C3F
:1019AE00C300000000C3330FFF0F33C3C03CC3039B
:1019BE00FF0303FF0000FC0CFC00000FF00F000003
:1019CE00000000C03F00000000FF000000000C0CF3
:1019DE00CF0F0CFC0C0CCC0F3C00000CCCFF0C0CF5
:1019EE00FC0000003FC03F00003F00300F000F031F
:1019FE00300F000F3000300C030000000030300FAD
:101A0E00000000000C030030303F000000030C000B
:101A1E000030300C0F030C3000300C030C30000083
:101A2E000CF00000F03030300C0C0C0C00000000FC
:101A3E0000FC0C0C0C0C0C0C0C0C0CFC0000000034
:101A4E000000000000000000000000000000000088
:101A5E0000000000303030F00000FF0CCC0C0C0CFD
:101A6E00CC3C0000000000FF0000FF030303FF005A
:101A7E0000FF000000000000000000000000000059
:101A8E0000000000000000000000000000FF00C089
:101A9E003F00C0330C33C0000000000000FF000008
:101AAE003F3030303F0000FF00000000000000001B
:101ABE000000000000000000000000000000000018
:101ACE0000300C030C3330333030303030333000D4
:101ADE000000003F0C0C0C0C0C0C0C0C0C3F00000E
:101AEE0000000000000000000000000000000000E8
:101AFE000000000000000000FCCCCCCCCCCCCCCC48
:101B0E00FC000000C0C0C0C0C0CCF0C0C0C0C0C08F
:101B1E00C00030C00000FC0C0C0C0CFC00000000DF
:101B2E0000C0C0C0C0CCF0C0C0C0C0C0C0C0CFCC10
:101B3E00CCCCCCCCCCCCCFC0C000000000FCCCCCEC
:101B4E00CCCCCCFC0000000C30000000FFC3C3C3A3
:101B5E00C3FF0000000000FF0C0CFFCCCCCCCCFF70
:101B6E000C0C00FFCCCCCCFF003CCC0CCC3C0000D1
:101B7E0000FC0C0CCCCCCCCCCC0C0CFC0000F00F34
:101B8E0000FC0CFC0C0CFC0CFC00000000FF000C1C
:101B9E003CCC0C0CCC3C0C000C0F0C0C033F03305B
:101BAE000C030C303000003F00000F0C0C0C0F002B
:101BBE00303F000F0000303F303F30303F303F307D
:101BCE0000300F0030300C0C03030C0C30300000D2
:101BDE00FCCCCCCCCCCCCCCCFC0000000000FC006F
:101BEE00C0C0C0C0F0303000000030C00000FC0C9F
:101BFE000C0C0CFC0000000000C0C0C0C0CCF0C03B
:101C0E00C0C0C0C0C0C0CFCCCCCCCCCCCCCCCFC054
:101C1E00C00030FF0000FFC0C0C0FFC0C0C0000C3D
:101C2E0030000000FFC3C3C3C3FF0000000000FF6D
:101C3E000C0CFFCCCCCCCCFF0C0C00FFCCCCCCFFD6
:101C4E00003CCC0CCC3C000000FF0000FF00C000AC
:101C5E003FC000000000F00F00FC0CFC0C0CFC0C54
:101C6E00FC00000000FF000C3CCC0C0CCC3C0C002B
:101C7E000C0F0C0C033F03300C030C303000003FF4
:101C8E0000000F03000C30030C3F000F0000303F2C
:101C9E00303F30303F303F3000300F0030300C0CD2
:101CAE0003030C0C303000000CF00000F03030302C
:101CBE000C0C0C0C0000000000FC0C0C0C0C0C0CA2
:101CCE000C0C0CFC000000000000000000000000E6
:101CDE00000000000000000000000000303030F076
:101CEE000000FF0CCC0C0C0CCC3C0000000000FFE4
:101CFE000000FF030303FF0000FF000000000000D0
:101D0E0000000000000000000000000000000000C5
:101D1E000000000000FF00C03F00C0330C33C000C5
:101D2E000000000000FF00003F3030303F0000FF99
:101D3E000000000000000000000000000000000095
:101D4E00000000000000000000300C030C333033A4
:101D5E0030303030303330000000003F0C0C0C0CB3
:101D6E000C0C0C0C0C3F00000000000000000000EA
:101D7E00000000000000000000000000000000F065
:101D8E00FCFCFFFFFFFFFFFFFFFFFFFFFFFFFFFF5B
:101D9E00FFFFFFFFFFFFFCFCF000FFFFFFFF003C1B
:101DAE003C00FFFF3C3C3C3C3C3C3C3C3C3C3C3C1B
:101DBE003C3CFFFFFFFFFFFFFFFFFFFFFFFFFFFFAB
:101DCE00FFFFFFFFFFFFFFFFFFFFFFFFFFFFFFFF15
:101DDE00FFFFFFFFFFFF003C3C00FFFF3C3C3C3C95
:101DEE003C3C3C3C3C3C3C3C3C3CFFFFFFFFFFFF93
:101DFE00FFFFFFFFFFFFFFFFFFFFFFFFFFFFFFFFE5
:101E0E00FFFFFFFFFFFFFFFFFFFFFFFFFFFF003C96
:101E1E003C00FFFF3C3C3C3C3C3C3C3C3C3C3C3CAA
:101E2E003C3CFFFFFFFF000F3F3FFFFFFFFFFFFFA9
:101E3E00FFFFFFFFFFFFFFFFFFFFFFFFFFFF3F3F24
:101E4E000F0000F0FCFCFFFFFFFFFFFFFFFFFFFF97
:101E5E00FFFFFFFFFFFFFFFFFFFFFCFCF000FFFF98
:101E6E00FFFF00FFFFFFFFFFFFFFFFFFFFFFFFFF73
:101E7E00FFFFFFFFFFFFFFFFFFFFFFFFFFFF00FF63
:101E8E00FFFFFF0FF3FCFCFCF3CF3FFFFFFFFFFF55
:101E9E00FFFFFFFFFFFFFFFFFFFF00FFFF0FF0FF42
:101EAE00FFFFFFFFFFFFFFFCF3F3F3F3F3F3FFFF7F
:101EBE00FFFFFFFFFFFF00FF03FCFFFFFFFFFFFF22
:101ECE00FFFFFFFFFFFFFFFFFFFFFFFFFFFFFFFF14
:101EDE00FFFF00003F3F3F3F3F3F3F3F3F3F3F3F02
:101EEE003F3F3F3F3F3FFFFFFFFF000F3F3FFFFFE3
:101EFE00FFFFFFFFFFFFFFFFFFFFFFFFFFFFFFFFE4
:101F0E00FFFF3F3F0F0000F0FCFCFFFFFFFFFFFF56
:101F1E00FFFFFFFFFFFFFFFFFFFFFFFFFFFFFCFCC9
:101F2E00F000FFFFFFFFFFFFFFFFFFFFFFFFFFFFC1
:101F3E00FFFFFFFFFFFFFFFFFFFFFFFFFFFFFFFFA3
:101F4E00FFFFFFFFCFCF03030000CFCFCFCFCFCF09
:101F5E00CFCF3FFFFFFFFFFFFFFFFFFFFFFFFFFFA3
:101F6E00FFFFFFFFFCFCFFFFFFFFFFFFFFFFFF0078
:101F7E00FFFFFFFFFFFFFFFFFFFFFFFFF3F3F3F393
:101F8E00F3F3F3F3F3F3F3F3F3F3FCFFFFFFFFFFCE
:101F9E00FFFFFFFFFFFFFFFFFFFFFFFFFFFFFFFF43
:101FAE00FFFFFFFFFFFFFFFFFFFFFFFFFFFF000F22
:101FBE003F3FFFFFFFFFFFFFFFFFFFFFFFFFFFFFA3
:101FCE00FFFFFFFFFFFF3F3F0F0000F00C0C03036E
:101FDE0003030303030303030303030303030303C3
:101FEE0003030C0CF000FF000000FFC3C3FF000052
:101FFE00C3C3C3C3C3C3C3C3C3C3C3C3C3C3000029
:10200E0000FFFF00000000000000000000000000C4
:10201E0000000000000000000000000000FFFF00B4
:10202E000000FFC3C3FF0000C3C3C3C3C3C3C3C306
:10203E00C3C3C3C3C3C3000000FFFF000000000002
:10204E000000000000000000000000000000000082
:10205E000000000000FFFF000000FFC3C3FF0000F0
:10206E00C3C3C3C3C3C3C3C3C3C3C3C3C3C30000B8
:10207E0000FF000F3030C0C0C0C0C0C0C0C0C0C064
:10208E00C0C0C0C0C0C0C0C0C0C030300F0000F063
:10209E000C0C0303030303030303030303030303F0
:1020AE000303030303030C0CF000FF000000FF000A
:1020BE000000000000000000000000000000000012
:1020CE000000000000FFFF000000FF00000000F015
:1020DE000C0303030C30C0000000000000000000E1
:1020EE0000FFFF000000FF0000F00F0000000000E6
:1020FE00000000030C0C0C0C0C0C000000FFFF0089
:10210E000000FF00FC0300000000000000000000C3
:10211E00000000000000000000FFFF000000FFFFB5
:10212E00C0C0C0C0C0C0C0C0C0C0C0C0C0C0C0C0A1
:10213E00C0C0000000FF000F3030C0C0C0C0C0C023
:10214E00C0C0C0C0C0C0C0C0C0C0C0C0C0C03030A1
:10215E000F00000CF000000C30000000300C0000EE
:10216E0000C03C00C000F03030F03030F000000015
:10217E00C03CC0C0C0CCF0C0C0C0C00000C0C0F0E9
:10218E00CCC0C0C0C0C000003030F00000C3C3C31C
:10219E00FFC3C3C300000C0FCC3C0300FFC0C0FF45
:1021AE00C0C0FF00300CFF0000CCCCCCCCCCCCCCD3
:1021BE00000000FFCCCCCCCCCCCCCCFF000000007F
:1021CE00FF0030303030FF30303030000C0F0C0C50
:1021DE000C00FF0000FF0000FF000000FF0000FCED
:1021EE000C0C0C0C0CFC0000000FCC0C0C3CCC0CA2
:1021FE000C0FC00000000F03000000003F000000A5
:10220E0000000C0C0C0303003F0C0C0F0C0C3F00D9
:10221E0000003F00003F0C0C0C0C0C3F00300F0078
:10222E000F30303033303C00000F0030C00000FC67
:10223E000C0C0C0CFC0000000000C0C0C0C0CCF0A8
:10224E00C0C0C0C0C00000000000FC0000FC0000C8
:10225E0000000000C03C00C0000000FC000C30007C
:10226E000C30000000FFC3C3C3C3FF00000000001A
:10227E00FF0C0CFFCCCCCCCCFF0C0C00FF030303EB
:10228E00FF0303FF030303FF000C0FCC3C03000C02
:10229E000CFF03C3C3C000F00F00FC0CFC0C0CFCC5
:1022AE000CFC00000000FF000C3CCC0C0CCC3C0CD9
:1022BE000000FF030303FF0303FF030303FF000CF0
:1022CE000F0C0C0C0003033FC3300CC00F0000308A
:1022DE003F303F30303F303F3000300F0030300C59
:1022EE000C03030C0C3030003F0C0C0C0F0C0C0FBD
:1022FE000C0C0C3F000C0C0C0303000C0C03000325
:10230E000C3F00000CF00000F03030300C0C0C0CC8
:10231E000000000000FC0C0C0C0C0C0C0C0C0CFC4B
:10232E00000000000000000000000000000000009F
:10233E000000000000000000303030F00000FF0C04
:10234E00CC0C0C0CCC3C0000000000FF0000FF0386
:10235E000303FF0000FF000000000000000000006B
:10236E00000000000000000000000000000000005F
:10237E0000FF00C03F00C0330C33C000000000005F
:10238E0000FF00003F3030303F0000FF0000000033
:10239E00000000000000000000000000000000002F
:1023AE000000000000300C030C333033303030307E
:1023BE00303330000000003F0C0C0C0C0C0C0C0CDD
:1023CE000C3F0000000000000000000000000000B4
:1023DE0000000000000000000000F0FCFFFFFFFF07
:1023EE00FFFFFF0F030303030CF01F7FFFFFFFFF31
:1023FE00FFFFFFE080808080601FF00CC3F3F3C30B
:10240E0003030303030303030CF00F30C3CFCFC347
:10241E00C0C0C0C0C0C0C0C0300F3F000000000030
:10242E00000000000000000000000000000000009E
:10243E00000000000000000000000000000000008E
:10244E00000000000000000000000000000000007E
:10245E00000000000000000000000000000000006E
:10246E00000000000000000000000000000000005E
:10247E00000000000000000000000000000000004E
:10248E00003F0000000000000000000000000000FF
:10249E00000000000000000000000000000000002E
:1024AE00000000000000000000000000000000001E
:1024BE00000000000000000000000000000000000E
:1024CE0000000000000000000000000000000000FE
:1024DE0000000000000000000000000000000000EE
:1024EE0000000000000000003F000000000000009F
:1024FE0000000000000000000000000000000000CE
:10250E0000000000000000000000000000000000BD
:10251E0000000000000000000000000000000000AD
:10252E00000000000000000000000000000000009D
:10253E00000000000000000000000000000000008D
:10254E000000000000000000000000000000003F3E
:10255E00000000000000000000000000000000006D
:10256E00000000000000000000000000000000005D
:10257E00000000000000000000000000000000004D
:10258E00000000000000000000000000000000003D
:10259E00000000000000000000000000000000002D
:1025AE00000000000000000000000000000000001D
:1025BE000000000000003F000000000000000000CE
:1025CE0000000000000000000000000000000000FD
:1025DE0000000000000000000000000000000000ED
:1025EE0000000000000000000000000000000000DD
:1025FE0000000000000000000000000000000000CD
:10260E0000000000000000000000000000000000BC
:10261E00000000000000000000000000003F00006D
:10262E00000000000000000000000000000000009C
:10263E00000000000000000000000000000000008C
:10264E00000000000000000000000000000000007C
:10265E00000000000000000000000000000000006C
:10266E00000000000000000000000000000000005C
:10267E00000000000000000000000000000000004C
:10268E00000000003F0000000000000000000000FD
:10269E00000000000000000000000000000000002C
:1026AE00000000000000000000000000000000001C
:1026BE00000000000000000000000000000000000C
:1026CE0000000000000000000000000000000000FC
:1026DE0000000000000000000000000000000000EC
:1026EE000000000000000000000000FFC0C0C0C0DD
:1026FE00C0C0C000C0C0C0C0C0C0C000C0C0C0C04C
:10270E00C0C0C000C0C0C0C0C0C0C000C0C0C0C03B
:10271E00C0C0C000C0C0C0C0C0C0C000C0C0C0C02B
:10272E00C0C0C000C0C0C0C0C0C0C000C0C0C0C01B
:10273E00C0C0C000C0C0C0C0C0C0C000C0C0C0C00B
:10274E00C0C0C000C0C0C0C0C0C0C000C0C0C0C0FB
:02275E00C0C0F9
:10398D004205D701F4420408012C4205D90000423A
:10399D0005DB00004205BA00004205D0015E42057C
:1039AD00CE00014205D4000A4205CA00144205C8E2
:1039BD00001E4205CC00004207DB00004205C2009C
:1039CD000042040200004205D200004205BC000086
:1039DD0044040C000000004405C400000000619088
:1039ED00064600000000000000000000000000007E
:1039FD0000000000000000000000000000000000BA
:103A0D0000000000000000000000000000000000A9
:103A1D000000000000000000000000000000000099
:103A2D000000000000000000000000000000000089
:103A3D000000000000000000000000000000000079
:103A4D000000000000000000000000000000000069
:103A5D000000000000000000000000000000000059
:103A6D000000000000000000000000000000000049
:103A7D000000000000000000000000000000000039
:103A8D000000000000000000000000000000000029
:103A9D000000000000000000000000000000000019
:103AAD000000000000000000000000000000000009
:103ABD0000000000000000000000000000000000F9
:103ACD0000000000000000000000000000000000E9
:103ADD0000000000000000000000000000000000D9
:103AED0000000000000000000000000000000000C9
:103AFD0000000000000000000000000000000000B9
:103B0D0000000000000000000000000000000000A8
:103B1D000000000000000000000000000000000098
:103B2D000000000000000000000000000000000088
:103B3D000000000000000000000000000000000078
:103B4D000000000000000000000000000000000068
:103B5D000000000000000000000000000000000058
:103B6D000000000000000000000000000000000048
:103B7D0000004407D743480000619004280000006E
:103B8D000000000000000000000000000000000028
:103B9D000000000000000000000000000000000018
:103BAD000000000000000000000000000000000008
:103BBD0000000000000000000000000000000000F8
:103BCD0000000000000000000000000000000000E8
:103BDD0000000000000000000000000000000000D8
:103BED0000000000000000000000000000000000C8
:103BFD0000000000000000000000000000000000B8
:103C0D0000000000000000000000000000000000A7
:103C1D000000000000000000000000000000000097
:103C2D000000000000000000000000000000000087
:103C3D000000000000000000000000000000000077
:103C4D000000000000000000000000000000000067
:103C5D000000000000000000000000000000000057
:103C6D000000000000000000000000000000000047
:103C7D000000000000000000000000000000000037
:103C8D000000000000000000000000000000000027
:103C9D000000000000000000000000000000000017
:103CAD000000000000000000000000000000000007
:103CBD0000000000000000000000000000000000F7
:103CCD0000000000000000000000000000000000E7
:103CDD0000000000000000000000000000000000D7
:103CED0000000000000000000000000000000000C7
:103CFD0000000000000000000000000000000000B7
:103D0D00000000000000000000000000004404114D
:103D1D00342BCC77440415BA6A76D74404193FF492
:103D2D00F36C44041DC4C03F304405BE00000000C8
:103D3D0041042600410410004107D6004104270428
:103D4D004105D60441064403410421034207E30023
:103D5D000042040A00004204060000420404000070
:103D6D004207E100004207DF0000606505DF00004B
:103D7D000000000000000000000000000000000036
:103D8D000000000000000000000000000000000026
:103D9D000000000000000000000000000000000016
:103DAD000000000000000000000000000000000006
:103DBD0000000000000000000000000000000000F6
:103DCD0000000000000000000000000000000000E6
:103DDD0000000041064564C180C18CC183C18BC107
:013DED008154
:0871C7009007E5EFF0A3EDF0E5
:1071CF007C007D0AAF03AE021253C4A3EDF07C0026
:1071DF007D0AAF03AE021253C47C007D0A1253C462
:1071EF00A3EDF0AE02AF037C007D641253C47C00AC
:1071FF007D0A1253C4AF05EF75F060A4240EF97425
:10720F000035F0FA9007F474FFF0A3EAF0A3E9F069
:10721F009007E5E0FFA3E0FD9007F37430F07B10DB
:10722F00126FDE9007E5E02410F09007E8E075F0AC
:10723F0060A4240EF9740035F0FA9007F474FFF08F
:10724F00A3EAF0A3E9F09007E5E0FFA3E0FD9007C4
:10725F00F37430F07B10126FDE9007E5E02410F02E
:10726F009007E7E075F060A4240EF9740035F0FA8A
:10727F009007F474FFF0A3EAF0A3E9F09007E5E0BC
:0F728F00FFA3E0FD9007F37430F07B10026FDE79
:086EE4009007E5EFF0A3EDF0CB
:106EEC007C007D0AAF03AE021253C49007EAEDF0AA
:106EFC007C007D0AAF03AE021253C47C007D0A12E3
:106F0C0053C4A3EDF0AE02AF037C007D641253C4F6
:106F1C00EF75F018A424CEF9740335F0FA9007F449
:106F2C0074FFF0A3EAF0A3E9F09007E5E0FFA3E01B
:106F3C00FD9007F37418F07B08126FDE9007E5E004
:106F4C002408F09007EBE075F018A424CEF9740334
:106F5C0035F0FA9007F474FFF0A3EAF0A3E9F0908F
:106F6C0007E5E0FFA3E0FD9007F37418F07B08122F
:106F7C006FDE9007E5E02408F09007EAE075F01862
:106F8C00A424CEF9740335F0FA9007F474FFF0A33F
:106F9C00EAF0A3E9F09007E5E0FFA3E0FD9007F32A
:106FAC007418F07B08126FDE9007E9E060239007FD
:106FBC00E5E02408F0E0FFA3E0FD9007F37418F07F
:106FCC00A374FFF0A37405F0A37403F07B0B126F92
:016FDC00DED6
:016FDD002291
:085E19009007E5EFF0A3EDF0A6
:105E2100E4FFFE7D207C41A3E0F8A3E0F9A3E0FAC2
:105E3100A3E0FB1252224003025F80E4FFFE7DC813
:105E41007C429007E7E0F8A3E0F9A3E0FAA3E0FBC6
:105E510012507C1252D99007EEEEF0A3EFF09007AA
:105E6100EEE0FAA3E0FB7C007D64FFAE021253C4B6
:105E71009007EBEFF07C007D0AAF03AE021253C432
:105E81007C007D0A1253C4A3EDF09007EEE0FEA35F
:105E9100E0FF7C007D0A1253C49007EDEDF09007FE
:105EA100EBE075F018A424CEF9740335F0FA9007ED
:105EB100F474FFF0A3EAF0A3E9F09007E5E0FFA393
:105EC100E0FD9007F37418F07B08126FDE9007E590
:105ED100E02408F0E0FFA3E0FD9007F37418F0A3BD
:105EE10074FFF0A37405F0A3743CF07B02126FDE23
:105EF1009007E5E02402F09007ECE075F018A42487
:105F0100CEF9740335F0FA9007F474FFF0A3EAF0C8
:105F1100A3E9F09007E5E0FFA3E0FD9007F3741813
:105F2100F07B08126FDE9007E5E02408F09007EDA2
:105F3100E075F018A424CEF9740335F0FA9007F453
:105F410074FFF0A3EAF0A3E9F09007E5E0FFA3E016
:105F5100FD9007F37418F07B08126FDE9007E5E0FF
:105F61002408F0E0FFA3E0FD9007F37418F0A37498
:105F7100FFF0A37405F0A37424F07B08126FDEE434
:105F8100FFFE7D207C419007E7E0F8A3E0F9A3E064
:105F9100FAA3E0FB12522250030260E1E4FFFE7D0E
:105FA100207C419007E7E0F8A3E0F9A3E0FAA3E041
:105FB100FB12507C1252D99007EEEEF0A3EFF09055
:105FC10007EEE0FAA3E0FB7C007D64FFAE02125312
:105FD100C49007EBEFF07C007D0AAF03AE021253D1
:105FE100C47C007D0A1253C4A3EDF09007EEE0FEDD
:105FF100A3E0FF7C007D0A1253C49007EDEDF09001
:1060010007EBE075F018A424CEF9740335F0FA908B
:1060110007F474FFF0A3EAF0A3E9F09007E5E0FFCD
:10602100A3E0FD9007F37418F07B08126FDE900770
:10603100E5E02408F09007ECE075F018A424CEF90F
:10604100740335F0FA9007F474FFF0A3EAF0A3E9C2
:10605100F09007E5E0FFA3E0FD9007F37418F07BF3
:1060610008126FDE9007E5E02408F0E0FFA3E0FDF1
:106071009007F37418F0A374FFF0A37405F0A374F0
:106081003CF07B02126FDE9007E5E02402F09007FE
:10609100EDE075F018A424CEF9740335F0FA9007F9
:1060A100F474FFF0A3EAF0A3E9F09007E5E0FFA3A1
:1060B100E0FD9007F37418F07B08126FDE9007E59E
:1060C100E02408F0E0FFA3E0FD9007F37418F0A3CB
:1060D10074FFF0A37405F0A37424F07B08126FDE43
:0160E100229C
:0B6B6C009007E5EFF0A3EDF0A3EBF0C5
:106B7700A3E0601075F035A4FFAEF07C007D6412D1
:106B870053C4EFF09007E5E0FFA3E0FD9007F3742F
:106B970010F0A374FFF0A37405F0A37442F07B37E1
:106BA700126FDE9007E7E0146074046003026CA6BE
:106BB7009007E6E0FD9007F37410F0A374FFF0A3CD
:106BC7007405F0A374B0F07B08E4FF126FDE900742
:106BD700E8E07003026CA6E4A3F09007E8E014FF76
:106BE700A3E0FEC39F50289007E5E02E04FBFFA318
:106BF700E075F008A4FE2402FDEE240D9007EFF0E7
:106C0700A37401F0125B329007E9E004F080CB90A7
:106C170007E8E0FF9007E5E02FFBFFA3806A9007F6
:106C2700E6E0FD9007F37410F0A374FFF0A374057A
:106C3700F0A374C0F07B087F78126FDE9007E8E05E
:106C4700605DE4A3F09007E8E014FFA3E0FEC39FB4
:106C57005028C374769EFBFF9007E6E075F008A402
:106C6700FE2402FDEE240D9007EFF0A37401F0124D
:106C77005B329007E9E004F080CB9007E8E0FFC3C0
:106C870074779FFBFF9007E6E075F008A4FE2404E5
:0F6C9700FDEE240B9007EFF0A37401F0125B32B7
:016CA60022CB
:1060E2009007E5EFF0A3EDF0A3EBF06011E075F09F
:1060F20030A4FFAEF07C007D641253C4EFF0900731
:10610200EAE0FEA3E0FFD39007E9E09F9007E8E012
:106112009E9007E7E0FF9007E5E0500302621C2F24
:1061220024FEFBFFA3E0FE2406FDEE24099007EF08
:10613200F0A37401F0125B329007E7E0FF9007E5ED
:10614200E02F14FBFFA3E0FE2404FDEE240B9007D6
:10615200EFF0A37401F0125B329007E7E0FF9007C3
:10616200E5E02F14FBFFA3E0FE2406FDEE240990D8
:1061720007EFF0E4A3F0125B329007E7E0FF90072D
:10618200E5E02FFBFFA3E0FE2402FDEE240D9007C5
:10619200EFF0A37401F0125B329007E7E0FF900783
:1061A200E5E02FFBFFA3E0FE2404FDEE240B9007A5
:1061B200EFF0E4A3F0125B329007E7E0FF9007E50F
:1061C200E02F04FBFFA3E0FE2404FDEE240B900766
:1061D200EFF0A37401F0125B329007E7E0FF900743
:1061E200E5E02F04FBFFA3E0FE2406FDEE24099068
:1061F20007EFF0E4A3F0125B329007E7E0FF9007AD
:10620200E5E02F2402FBFFA3E0FE2406FDEE2409B5
:106212009007EFF0A374010263122F24FEFBFFA389
:10622200E0FE2406FDEE24099007EFF0E4A3F0124D
:106232005B329007E7E0FF9007E5E02F14FBFFA336
:10624200E0FE2404FDEE240B9007EFF0E4A3F0122D
:106252005B329007E7E0FF9007E5E02F14FBFFA316
:10626200E0FE2406FDEE24099007EFF0A37401F08E
:10627200125B329007E7E0FF9007E5E02FFBFFA3F8
:10628200E0FE2402FDEE240D9007EFF0E4A3F012ED
:106292005B329007E7E0FF9007E5E02FFBFFA3E00A
:1062A200FE2404FDEE240B9007EFF0A37401F0121C
:1062B2005B329007E7E0FF9007E5E02F04FBFFA3C6
:1062C200E0FE2404FDEE240B9007EFF0E4A3F012AD
:1062D2005B329007E7E0FF9007E5E02F04FBFFA3A6
:1062E200E0FE2406FDEE24099007EFF0A37401F00E
:1062F200125B329007E7E0FF9007E5E02F2402FBF4
:10630200FFA3E0FE2406FDEE24099007EFF0E4A3CC
:05631200F0125B3222D5
:0E6317009007E5EFF0A3EDF0A3EAF0A3EBF0A2
:10632500A3E0640360030263E09007E7E0FAA3E0FB
:10633500FB7C007D64FFAE021253C49007EAEFF0C8
:106345007C007D0AAF03AE021253C47C007D0A12A5
:1063550053C4A3EDF09007E7E0FEA3E0FF7C007DCA
:106365000A1253C49007ECEDF09007EAE075F018B7
:10637500A424CEF9740335F0FA9007F474FFF0A362
:10638500EAF0A3E9F09007E5E0FFA3E0FD9007F34D
:106395007418F07B08126FDE9007E5E02408F09092
:1063A50007EBE075F018A424CEF9740335F0FA90E4
:1063B50007F474FFF0A3EAF0A3E9F09007E5E0FF26
:1063C500A3E0FD9007F37418F07B08126FDE9007C9
:1063D500E5E02408F09007EC0264E59007E9E06445
:1063E5000460030265119007E7E0FAA3E0FB7C0374
:1063F5007DE8FFAE021253C49007EAEFF07C007D02
:1064050064AF03AE021253C47C007D0A1253C4A3C9
:10641500EDF09007E7A3E07C007D0AFFAE02125382
:10642500C47C007D0A1253C49007ECEDF07C007D1E
:106435000AAF03AE021253C4A3EDF09007EAE0756C
:10644500F018A424CEF9740335F0FA9007F474FF1C
:10645500F0A3EAF0A3E9F09007E5E0FFA3E0FD90E3
:1064650007F37418F07B08126FDE9007E5E0240847
:10647500F09007EBE075F018A424CEF9740335F01D
:10648500FA9007F474FFF0A3EAF0A3E9F09007E5AA
:10649500E0FFA3E0FD9007F37418F07B08126FDEB0
:1064A5009007E5E02408F09007ECE075F018A424C7
:1064B500CEF9740335F0FA9007F474FFF0A3EAF00F
:1064C500A3E9F09007E5E0FFA3E0FD9007F374185A
:1064D500F07B08126FDE9007E5E02408F09007EDE9
:1064E500E075F018A424CEF9740335F0FA9007F49A
:1064F50074FFF0A3EAF0A3E9F09007E5E0FFA3E05D
:0C650500FD9007F37418F07B08126FDEA5
:016511002267
:104A11007B017A0779E39007EAE4F0A37402F0E4FA
:104A2100FFFE1279A57B017A04790A9007EAE4F086
:104A3100A37402F07F00FE1279A57B017A04790646
:104A41009007EAE4F0A37402F07F04FE1279A57BDB
:104A5100017A0479049007EAE4F0A37402F07F0874
:104A6100FE1279A57B017A0779E19007EAE4F0A3C8
:104A71007402F07F007E041279A57B017A0779DF49
:104A81009007EAE4F0A37402F07404FFFE1279A522
:104A91007B017A0779D69007EAE4F0A304F07F005E
:104AA1007E061279A59007E4E0FE9007E3E07C0022
:104AB1002400FFEC3E900408F0A3EFF090040BE01B
:104AC100FE90040AE02400FFEC3E9005D4F0A3EF31
:104AD100F0900407E0FE900406E02400FFEC3E9015
:104AE10005CAF0A3EFF0900405E0FE900404E02471
:104AF10000FFEC3E9005C8F0A3EFF09007E2E0FE66
:104B01009007E1E02400FFEC3E9005D0F0FCA3EF1C
:104B1100F0FD9007E0E0FE9007DFE07A002400FF5F
:104B2100EA3E9005CEF0A3EFF0D3ED945EEC940154
:104B3100400AA37401F0A3745EF08015C39005D1FF
:104B4100E094C89005D0E094005006E4F0A374C846
:104B5100F09005CEE0FEA3E0D394C8EE94004002AD
:104B61008006C3EE94005007E49005CEF0A3F090C8
:104B710005D0E0FEA3E0FF900408E0FCA3E0FDD334
:104B81009FEC9E4002800F9005CEE0FEA3E0FFC3A4
:104B9100ED9FEC9E5008900408EEF0A3EFF0900515
:104BA100D4E0FEA3E0D394F4EE9401400B9005D43D
:104BB100E4F0A37464F0800DC3EE94005007E49018
:104BC10005D4F0A3F09005CAE0FEA3E0D394F4EE7F
:104BD1009401400B9005CAE4F0A37464F0800DC306
:104BE100EE94005007E49005CAF0A3F09005C8E0E8
:104BF100FEA3E0D394F4EE9401400B9005C8E4F0D9
:104C0100A37464F0800DC3EE94005007E49005C8CE
:104C1100F0A3F0900421E0FF24FEFE9007D6E0D33C
:104C21009E5006EFC394005005E49007D6F0E4F5DA
:104C3100927591FF75B2FF75B10CC2B4C2009004B8
:104C41002212549500000000127BCE12766E127B68
:104C510069D2AF90040CE0F8A3E0F9A3E0FAA3E075
:104C6100FBE4FFFE7DC87C42124F879005C41254BD
:104C710089E49005DDF0A3F0900645E0FFC39005BF
:104C8100DEE09F9005DDE094004003024D70E4FFFB
:104C9100FE1275BCAC06AD07E41252A0C004C005FB
:104CA100C006C0079005DDE0FEA3E07802C333CE65
:104CB10033CED8F92446F58274063EF583D007D069
:104CC10006D005D0041254897F017E001275BCC044
:104CD10006C007900411E0FCA3E0FDA3E0FEA3E001
:104CE100FF9007E7125489900415E0FCA3E0FDA3AF
:104CF100E0FEA3E0FF9007EB125489900419E0FC59
:104D0100A3E0FDA3E0FEA3E0FF9007EF125489901A
:104D1100041DE0FCA3E0FDA3E0FEA3E0FF9007F388
:104D2100125489D007D0061270D5AC06AD07E41233
:104D310052A0C004C005C006C0079005DDE0FEA377
:104D4100E07802C333CE33CED8F92428F582740437
:104D51003EF583D007D006D005D0041254899005C2
:104D6100DEE004F070069005DDE004F0024C79E429
:104D71009005DDF0A3F0900645E0FFC39005DEE06D
:104D81009F9005DDE0940050599005BEE0F8A3E046
:104D9100F9A3E0FAA3E0FBC000C001C002C0037F99
:104DA1000F7E001275BCAC06AD07E41252A0A80438
:104DB100A905AA06AB077FEC7E517D987C4512516F
:104DC10085D003D002D001D000124F8B9005BE12C6
:104DD10054899005DEE004F0709C9005DDE004F05C
:104DE10080949005BEE0FCA3E0FDA3E0FEA3E0FFFC
:104DF100C004C005C006C007900645E0FCE412529D
:104E0100A5A804A905AA06AB07D007D006D005D0EE
:104E1100041251859005BE125489E49005DDF0A37A
:104E2100F0900645E0FFC39005DEE09F9005DDE0D0
:104E310094004003024F14900422E0F8A3E0F9A388
:104E4100E0FAA3E0FBC000C001C002C0039005DD91
:104E5100E0FEA3E07802C333CE33CED8F92446F581
:104E61008274063EF583E0FCA3E0FDA3E0FEA3E02F
:104E7100FFE4FBFA79807845125185C004C005C072
:104E810006C007E4FFFE7DA07C419005BEE0F8A3CB
:104E9100E0F9A3E0FAA3E0FB12507CD003D002D0EA
:104EA10001D00012507CD003D002D001D000124FAB
:104EB1008B9004221254899007D7E0FCA3E0FDA354
:104EC100E0FEA3E0FFC004C005C006C0079005DDF9
:104ED100E0FEA3E07802C333CE33CED8F92428F51F
:104EE1008274043EF583E0F8A3E0F9A3E0FAA3E0BD
:104EF100FBD007D006D005D004124F8B9007D712F4
:104F010054899005DEE004F070069005DDE004F0C0
:104F1100024E22900422E0FCA3E0FDA3E0FEA3E008
:104F2100FFC004C005C006C007900645E0FCE412BE
:104F310052A5A804A905AA06AB07D007D006D0053B
:104F4100D0041251859004221254899007D7E0FCB5
:104F5100A3E0FDA3E0FEA3E0FFC004C005C006C0BE
:104F610007900645E0FCE41252A5A804A905AA068B
:104F7100AB07D007D006D005D0041251859007D7D2
:034F81000254894E
:107B3C00124A11900410E070031254F2900410E0F9
:087B4C00B401F012276080EB88
:03000B0002771960
:10771900C0E0C0F0C083C082C0D075D000C000C036
:1077290001C002C003C004C005C006C0079005B966
:10773900E004F070069005B8E004F09005B8E0FEAA
:10774900A3E0FF7C037DE81253C49005B8ECF0FE7A
:10775900A3EDF0FF7C037DE81253C4ED4C7007C222
:107769000A300002D2079005B8E0FAA3E0FB7C00DA
:107779007D0AFFAE021253C4ED4C7002C202C390DF
:1077890005CDE09B9005CCE09A4007300004D2B4C7
:107799008002C2B4127847D007D006D005D004D0F1
:1077A90003D002D001D000D0D0D082D083D0F0D085
:0277B900E032BC
:1078470020B21630B3132004109005DAE004F0706C
:10785700069005D9E004F0D20820B31630B2132001
:1078670004109005DCE004F070069005DBE004F0FE
:10787700D20920B24320B3409005D7E0FEA3E0FF32
:10788700C39005DAE09F9005D9E09E502BC3900581
:10789700DCE09F9005DBE09E501EC209C208E4F0C1
:1078A700A3F09005D9F0A3F09005BBE004F07006B3
:0978B7009005BAE004F0D20422AD
:1065120020B2399005D7E0FEA3E0FFC39005DAE090
:106522009F9005D9E09E40249005D0E0FEA3E0FFB5
:10653200900409E09F900408E09E5042A3E004F01A
:106542007006900408E004F0C20C803230B22F30A2
:10655200082C9005D0E0FEA3E0FFC3900409E09F61
:10656200900408E09E5017A3E004F070069004081F
:10657200E004F0E49005D9F0A3F0C208C20C20B305
:106582003A9005D7E0FEA3E0FFC39005DCE09F90C0
:1065920005DBE09E40259005CEE0FEA3E0FFD39010
:1065A2000409E09F900408E09E4045A3E024FFF028
:1065B200900408E034FFF0C20C803530B332300969
:1065C2002F20062C9005CEE0FEA3E0FFD390040915
:1065D200E09F900408E09E4017A3E024FFF090049F
:1065E20008E034FFF0E49005DBF0A3F0C209C20C2E
:1065F20020B24720B3449005D7E0FEA3E0FFC3904A
:1066020005BBE09F9005BAE09E402F30042C300578
:1066120029900410E070047F0180027F0090041032
:10662200EFF0C200C2B4C204E49005BAF0A3F0C213
:10663200059007DBF0A304F0804430B34130B23E52
:1066420030043B9005D7E0FEA3E0FFC39005BBE01A
:106652009F9005BAE09E5026300523B2009007DBDA
:10666200E4F0A304F0A20092B4E49005D2F0A3F007
:106672009005CCF0A3F0C2049005BAF0A3F030B3B9
:106682005330B250E49005BAF0A3F0C204D20590A0
:1066920005D9F0A3F0A3F0A3F0C208C209200C347C
:1066A200900408E0FEA3E09007E3F0EEA3F0E4FF1D
:1066B200FE127B7C7B017A0779E39007EAE4F0A380
:1066C2007402F0E4FFFE12796CE49007E4F09007A4
:0A66D200E3F0D20C300602C20622EB
:1054F200127B083002030255B6900426E004F0E065
:10550200FF900645E0FEEF8EF084900426E5F0F071
:10551200E4FFFE1275BCAC06AD07E41252A0900483
:1055220026E075F004A42446F582E5F03406F583FE
:105532001254897F017E001275BCC006C007900418
:1055420011E0FCA3E0FDA3E0FEA3E0FF9007E71259
:105552005489900415E0FCA3E0FDA3E0FEA3E0FF64
:105562009007EB125489900419E0FCA3E0FDA3E03C
:10557200FEA3E0FF9007EF12548990041DE0FCA304
:10558200E0FDA3E0FEA3E0FF9007F3125489D007E9
:10559200D0061270D5AC06AD07E41252A0900426D4
:1055A200E075F004A42428F582E5F03404F58312B2
:1055B2005489D2029007D71254950000000090043B
:1055C20022125495000000009005BE12549500006E
:1055D2000000E49005DDF0A3F0900645E0FFC390E3
:1055E20005DEE09F9005DDE0940050599005BEE095
:1055F200F8A3E0F9A3E0FAA3E0FBC000C001C002F7
:10560200C0037F0F7E001275BCAC06AD07E41252D8
:10561200A0A804A905AA06AB077FEC7E517D987C61
:1056220045125185D003D002D001D000124F8B9089
:1056320005BE1254899005DEE004F070069005DD87
:10564200E004F080949005BEE0FCA3E0FDA3E0FE40
:10565200A3E0FFC004C005C006C007900645E0FCF9
:10566200E41252A5A804A905AA06AB07D007D006E2
:10567200D005D0041251859005BE125489E49005DC
:10568200DDF0A3F0900645E0FFC39005DEE09F90B9
:1056920005DDE094004003025778900422E0F8A36D
:1056A200E0F9A3E0FAA3E0FBC000C001C002C0031E
:1056B2009005DDE0FEA3E07802C333CE33CED8F905
:1056C2002446F58274063EF583E0FCA3E0FDA3E0E8
:1056D200FEA3E0FFE4FBFA79807845125185C0040D
:1056E200C005C006C007E4FFFE7DA07C419005BE58
:1056F200E0F8A3E0F9A3E0FAA3E0FB12507CD003A8
:10570200D002D001D00012507CD003D002D001D000
:1057120000124F8B9004221254899007D7E0FCA309
:10572200E0FDA3E0FEA3E0FFC004C005C006C00781
:105732009005DDE0FEA3E07802C333CE33CED8F984
:105742002428F58274043EF583E0F8A3E0F9A3E08F
:10575200FAA3E0FBD007D006D005D004124F8B90FD
:1057620007D71254899005DEE004F070069005DD3B
:10577200E004F0025686900422E0FCA3E0FDA3E0E0
:10578200FEA3E0FFC004C005C006C007900645E0C6
:10579200FCE41252A5A804A905AA06AB07D007D0BB
:1057A20006D005D004125185900422125489900724
:1057B200D7E0FCA3E0FDA3E0FEA3E0FFC004C00528
:1057C200C006C007900645E0FCE41252A5A804A951
:1057D20005AA06AB07D007D006D005D00412518522
:1057E2009007D7125489E4FFFE7DC87C439007D707
:1057F200E0F8A3E0F9A3E0FAA3E0FB125222600270
:105802005018E4FFFEFDFC9007D7E0F8A3E0F9A3EF
:10581200E0FAA3E0FB125222500A9007D7125495E5
:1058220000000000300705126874C2079007D6E036
:105832007005125849800A9007D6E0B40103126637
:07584200DC127AD2026512AC
:1030800030B2030231C29005D7E0FEA3E0FFC39047
:1030900005DAE09F9005D9E09E50030231C2900707
:1030A000DBE0FEA3E0FF9464EE64809480500302B2
:1030B0003143EF946EEE6480948040030231437C90
:1030C000007D0A125419EC6003023386ED14602D62
:1030D00014604D24026003023386C39005D5E0944A
:1030E000F49005D4E094014003023386A3E004F099
:1030F00070069005D4E004F0C203023386C3900545
:10310000CBE094F49005CAE094014003023386A317
:10311000E004F070069005CAE004F0C203023386B2
:10312000C39005C9E094F49005C8E09401400302FF
:103130003386A3E004F070069005C8E004F0C203F3
:103140000233869007DBE0FEA3E0FFC394C8EE6481
:103150008094805003023386EF94D2EE6480948092
:1031600040030233867C007D0A125419EC6003028E
:103170003386ED146029046003023386C39005D1C1
:10318000E0945E9005D0E094014003023386A3E012
:1031900004F070069005D0E004F0C20B023386C341
:1031A0009005CFE094C89005CEE094004003023330
:1031B00086A3E004F070069005CEE004F0C20B0296
:1031C000338620B203023386200803023386900739
:1031D000DBE0FEA3E0FFC39464EE64809480500EB5
:1031E000E004F070069007DBE004F00232F2C3EF77
:1031F0009464EE648094805003023289EF946EEE02
:103200006480948040030232897C007D0A12541944
:10321000EC60030232F2ED14602D14604D24026064
:10322000030232F2C39005D5E094F49005D4E09403
:103230000140030232F2A3E004F070069005D4E0EE
:1032400004F0C2030232F2C39005CBE094F490057F
:10325000CAE0940140030232F2A3E004F070069049
:1032600005CAE004F0C2030232F2C39005C9E0943B
:10327000F49005C8E094015079A3E004F070069042
:1032800005C8E004F0C20380699007DBE0FEA3E01C
:10329000FFC394C8EE648094804057EF94D2EE64EC
:1032A000809480504D7C007D0A125419EC7043EDDF
:1032B00014602204703CC39005D1E0945E9005D068
:1032C000E09401502DA3E004F070069005D0E004D6
:1032D000F0C20B801DC39005CFE094C89005CEE0EE
:1032E0009400500EA3E004F070069005CEE004F0C8
:1032F000C20B900427E02401FFE433FE9007DBE0DB
:10330000FCA3E0FDB5070EECB5060A9007DBE4F080
:10331000A304F080689005D6E0FF240AFBE433FAAA
:10332000EDB50314ECB50210C39007DCE09FF090FC
:1033300007DBE09400F08045900644E0F92414FF98
:10334000E433FE9007DBE0FCA3E0FDB50706ECB537
:1033500006028019900421E0241EFFE433FE90074A
:10336000DBE0FCA3E0FDB50714ECB50610E9FFC3F4
:10337000ED9FFEEC94009007DBF0A3CEF0E4900507
:10338000D9F0A3F0C20830B3030234B09005D7E0FF
:10339000FEA3E0FFC39005DCE09F9005DBE09E50BC
:1033A000030234B09007DBE0FEA3E0FF9464EE6418
:1033B0008094805003023438EF946EEE64809480E1
:1033C00050767C007D0A125419EC6003023625ED1C
:1033D00014602614603F24026003023625D3900552
:1033E000D5E094009005D4E094005003023625A364
:1033F000E024FFF09005D48036D39005CBE0940014
:103400009005CAE094005003023625A3E024FFF0A3
:103410009005CA801AD39005C9E094009005C8E0D1
:1034200094005003023625A3E024FFF09005C8E085
:1034300034FFF0C2030236259007DBE0FEA3E0FF75
:10344000C394C8EE648094805003023625EF94D272
:10345000EE6480948040030236257C007D0A12547D
:1034600019EC6003023625ED146022046003023675
:1034700025D39005D1E094C89005D0E09400500386
:10348000023625A3E024FFF09005D0801AD39005E2
:10349000CFE094009005CEE094005003023625A3BF
:1034A000E024FFF09005CEE034FFF0C20B02362599
:1034B00020B3030236252009030236259007DBE0FE
:1034C000FEA3E0FFC39464EE64809480500EE02479
:1034D000FFF09007DBE034FFF00235C6C3EF9464E1
:1034E000EE64809480407CEF946EEE648094805013
:1034F000727C007D0A125419EC60030235C6ED148B
:10350000602614603F240260030235C6D39005D5BF
:10351000E094009005D4E0940050030235C6A3E087
:1035200024FFF09005D48033D39005CBE094009035
:1035300005CAE0940050030235C6A3E024FFF090D2
:1035400005CA8017D39005C9E094009005C8E0949F
:10355000004073A3E024FFF09005C8E034FFF0C200
:103560000380639007DBE0FEA3E0FFC394C8EE6432
:103570008094804051EF94D2EE6480948050477CD8
:10358000007D0A125419EC703DED14601C04703675
:10359000D39005D1E094C89005D0E094004027A3D3
:1035A000E024FFF09005D08017D39005CFE0940081
:1035B0009005CEE09400400EA3E024FFF09005CEED
:1035C000E034FFF0C20B9007DBE0FEA3E0FF4E709B
:1035D0000F900427E0FD9007DBE4F0A3EDF0803CC2
:1035E000EF64094E70059005D680229007DBE0FE5F
:1035F000A3E0FF64134E700C900644E0FD9007DCDE
:10360000E02D8010EF641D4E7012900644E0FF9094
:1036100007DCE02FF09007DBE03400F0E49005DBFE
:10362000F0A3F0C20930B2030236D430B30302363D
:10363000D49005D7E0FEA3E0FFC39005BBE09F90C8
:1036400005BAE09E50030236D42004030236D4208B
:1036500005030236D49007DBE0FEA3E0FF940AEEF8
:103660006480948050519005CEE0FCA3E0FD90046E
:1036700008E0FAA3E0FBC39DEA9C5002800F90058E
:10368000D0E0FCA3E0FDD3EB9DEA9C400890040849
:10369000ECF0A3EDF0900410E070047D0180027D59
:1036A00000900410EDF0C206E49007DBF0A3F0C236
:1036B00000C2B4C20480127C007D0A125419900723
:1036C000DBEEF0A3EFF0C204E49005BAF0A3F0C281
:1036D0000502388620B30302388620B203023886FA
:1036E0002004030238869005D7E0FEA3E0FFC390D4
:1036F00005BBE09F9005BAE09E4003023886200596
:1037000003023886900427E0FF9007DBE0FCA3E08B
:10371000FD6F7001EC705A9005CEE0FEA3E0FF90C3
:103720000408E0FAA3E0FBC39FEA9E5002800F90DA
:1037300005D0E0FEA3E0FFD3EB9FEA9E4008900493
:1037400008EEF0A3EFF0900410E070047F01800217
:103750007F00900410EFF0C206E49007DBF0A3F0C6
:10376000C200C2B4C2049005BAF0A3F0C205023888
:103770007DC3ED9464EC64809480402D9007DBE081
:10378000FEA3E0FF7C007D0A125419AA04AB059049
:1037900007DBE0FEA3E0FF7C007D0A125419EF2B4B
:1037A000FFEE3A9007DB0238449007DBE0FEA3E02F
:1037B000FF640D4E6006EF64164E70159007DBE057
:1037C000FEA3E0FF7C007D0A1254199007DBEE8017
:1037D000739007DBE0FEA3E0FFC3940AEE648094DD
:1037E00080500D7C007D0A1253B29007DBEE8054AE
:1037F0009007DBE0FEA3E0FFC3941EEE648094809C
:103800004048EF9428EE64809480503E7C007D0A0E
:10381000125419900421E024FFFFE434FFFEED6F01
:103820007002EC6E600BAF059007D6EFF0C201801E
:103830004C9007DBE0FEA3E0FF7C007D0A125419E8
:103840009007DBEEF0A3EFF080339007DBE0FEA300
:10385000E0FF7C007D0A1254197C007D641253B293
:10386000AA06AB079007DBE0FEA3E0FF7D0A125437
:1038700019EB2DFEEA3C9007DBF0A3CEF0C204E486
:103880009005BAF0A3F020B30302398720B20302F7
:103890003987E49005BAF0A3F0C204D20520037280
:1038A0009005D4E0FEA3E090040AF0EEA3F09005AA
:1038B000CAE0FEA3E0900406F0EEA3F09005C8E095
:1038C000FEA3E0900404F0EEA3F07F007E02127BE2
:1038D0007C7B017A04790A9007EAE4F0A37402F091
:1038E0007F00FE12796C7B017A0479069007EAE486
:1038F000F0A37402F07F04FE12796C7B017A0479E4
:10390000049007EAE4F0A37402F07F08FE12796CD9
:10391000D203200B519005D0E0FEA3E09007E1F028
:10392000EEA3F09005CEE0FEA3E09007DFF0EEA35B
:10393000F07F007E04127B7C7B017A0779E190079F
:10394000EAE4F0A37402F07F007E0412796C7B013C
:103950007A0779DF9007EAE4F0A37402F07404FFB9
:10396000FE12796CD20B20011E7F007E06127B7C3A
:103970007B017A0779D69007EAE4F0A304F07F0090
:0D3980007E0612796CD201200602D20622CA
:10276000127B08123080C39007DCE0940A9007DBEC
:10277000E06480948050639007F37430F0A374FF9A
:10278000F0A3740DF0A3742AF07B117D017F6D120C
:102790006FDE9007F37430F0A374FFF0A3740CF0B5
:1027A000A374C4F07B117D017F02126FDE9007F3EA
:1027B0007440F09007DCE07F00FEEF24C4F974075A
:1027C0003EFA9007F474FFF0A3EAF0A3E9F07B204F
:1027D000E4FD7F30126FDE02307D9007DBE0FEA368
:1027E000E0FFC3940AEE64809480500302299AEFBC
:1027F0009414EE64809480400302299A9007F37445
:1028000030F0A374FFF0A3740DF0A3742AF07B11D1
:102810007D017F6D126FDE9007F37430F0A374FFBB
:10282000F0A3740CF0A374C4F07B117D017F02123D
:102830006FDE9007DBE0FEA3E0FF7C007D0A125410
:10284000197E007FD81253B274A42FF974173EFA80
:102850009007F474FFF0A3EAF0A3E9F09007F37493
:1028600020F07B36E4FD7F34126FDE9007DBE0FE64
:10287000A3E0FF7C007D0A1254199005D6E024FFE6
:10288000FFE434FFFEC3ED9FEE6480F8EC648098B3
:1028900050107E007FC41253B274842FF974113E1D
:1028A000802F9007DBE0FEA3E0FF7C007D0A12543E
:1028B000199005D6E0FF24FFFBE434FFFAEDB503E1
:1028C0002CECB50228EF75F0C4A424B0F9740D35D2
:1028D000F0FA9007F474FFF0A3EAF0A3E9F0900790
:1028E000F37438F07B1CE4FD7F16126FDEE4900574
:1028F000DDF0A3F09005D6E0FF9005DDE0FAA3E05F
:10290000FBC39FEA9400400302307D9007DBE0FEAA
:10291000A3E0FF7C007D0A125419EB6D7002EA6C93
:102920009005D6602FE024FFFDE434FFFC7E007F9D
:10293000481253C49005DDA3E0FEEF8EF0A42416E8
:10294000FF9007F37408F0A374FFF0A3740DF0A3D5
:1029500074F6802DE024FFFDE434FFFC7E007F4808
:102960001253C49005DDA3E0FEEF8EF0A42416FF01
:102970009007F37408F0A374FFF0A3740EF0A3742F
:1029800002F07B0C7D07126FDE9005DEE004F07034
:10299000069005DDE004F00228F49007DBE0FEA3DA
:1029A000E0FFC39414EE648094805003022B5AEF2E
:1029B000941EEE648094804003022B5A9007F374B7
:1029C00030F0A374FFF0A3740DF0A3742AF07B1110
:1029D0007D017F6D126FDE9007F37430F0A374FFFA
:1029E000F0A3740CF0A374C4F07B117D017F02127C
:1029F0006FDE9007DBE0FEA3E0FF7C007D0A12544F
:102A0000197E007FD81253B274042FF9741B3EFA5A
:102A10009007F474FFF0A3EAF0A3E9F09007F374D1
:102A200020F07B36E4FD7F34126FDE9007DBE0FEA2
:102A3000A3E0FF7C007D0A125419900644E024FFB5
:102A4000FFE434FFFEC3ED9FEE6480F8EC648098F1
:102A5000500F7E007FC41253B2741C2FF97416807D
:102A60002F9007DBE0FEA3E0FF7C007D0A125419E3
:102A7000900644E024FFFFE434FFFEEDB5072EECA2
:102A8000B5062A7E007FC41253B274D02FF9741396
:102A90003EFA9007F474FFF0A3EAF0A3E9F0900780
:102AA000F37438F07B1CE4FD7F16126FDEE49005B2
:102AB000DDF0A3F0900644E0FF9005DDE0FAA3E02E
:102AC000FBC39FEA9400400302307D9007DBE0FEE9
:102AD000A3E0FF7C007D0A125419EB6D7002EA6CD2
:102AE000900644602FE024FFFDE434FFFC7E007F6D
:102AF000481253C49005DDA3E0FEEF8EF0A4241627
:102B0000FF9007F37408F0A374FFF0A3740DF0A313
:102B100074F6802DE024FFFDE434FFFC7E007F4846
:102B20001253C49005DDA3E0FEEF8EF0A42416FF3F
:102B30009007F37408F0A374FFF0A3740EF0A3746D
:102B400002F07B0C7D07126FDE9005DEE004F07072
:102B5000069005DDE004F0022AB49007DBE0FEA356
:102B6000E0FFC3941EEE648094805003022D21D3B5
:102B7000EF9428EE648094804003022D219007F3A7
:102B80007430F0A374FFF0A3740DF0A3742AF07BEB
:102B9000117D017F6D126FDE9007F37430F0A37426
:102BA000FFF0A3740CF0A374C4F07B117D017F02CD
:102BB000126FDE9007DBE0FEA3E0FF7C007D0A12CF
:102BC00054197E007FD81253B274602FF974213EDD
:102BD000FA9007F474FFF0A3EAF0A3E9F09007F38A
:102BE0007420F07B36E4FD7F34126FDE9007DBE06B
:102BF000FEA3E0FF7C007D0A125419900421E0241A
:102C0000FFFFE434FFFEEDB50708ECB506047E00D7
:102C1000801C9007DBE0FEA3E0FF7C007D0A1254DD
:102C2000199007D6E07E00B50511EEB5040D7FC4FE
:102C30001253B2748C2FF9741D801C9007DBE0FED8
:102C4000A3E0FF7C007D0A1254197E007FC412535A
:102C5000B274D82FF9741F3EFA9007F474FFF0A3F2
:102C6000EAF0A3E9F09007F37438F07B1CE4FD7FF1
:102C700016126FDEE49005DDF0A3F0900421E0FF72
:102C80009005DDE0FAA3E0FBC39FEA940040030255
:102C9000307D9007DBE0FEA3E0FF7C007D0A12544C
:102CA00019EB6D7002EA6C900421602FE024FFFDA7
:102CB000E434FFFC7E007F481253C49005DDA3E09E
:102CC000FEEF8EF0A42416FF9007F37408F0A374AF
:102CD000FFF0A3740DF0A374F6802DE024FFFDE453
:102CE00034FFFC7E007F481253C49005DDA3E0FE54
:102CF000EF8EF0A42416FF9007F37408F0A374FF7E
:102D0000F0A3740EF0A37402F07B0C7D07126FDE4B
:102D10009005DEE004F070069005DDE004F0022C82
:102D20007B9007DBE0FEA3E0FFC39464EE64809435
:102D3000805003022ED3EF946EEE648094804003A3
:102D4000022ED39007F37430F0A374FFF0A3740E37
:102D5000F0A3740EF07B117D017F6D126FDE900782
:102D6000F37430F0A374FFF0A3740DF0A37490F02B
:102D70007B117D017F02126FDE9007DBE0FEA3E096
:102D8000FF7C007D0A1254197E007FC41253B27476
:102D9000742FF9740E3EFA9007F474FFF0A3EAF072
:102DA000A3E9F09007F37438F07B1CE4FD7F161262
:102DB0006FDE9007DBE0FEA3E0FF7C007D0A12548B
:102DC000197E007FD81253B274A42FF974173EFAFB
:102DD0009007F474FFF0A3EAF0A3E9F09007F3740E
:102DE00020F07B36E4FD7F34126FDE9007DBE0FEDF
:102DF000A3E0FF7C007D0A125419EC7029ED1460E9
:102E00000C14600E2402701E9005D480089005CA30
:102E100080039005C8E0FAA3E0FB9007E97404F092
:102E2000FD7F35126317E49005DDF0A3F09005D621
:102E3000E0FF9005DDE0FAA3E0FBC39FEA940040C9
:102E40000302307D9007DBE0FEA3E0FF7C007D0AFB
:102E5000125419EB6D7002EA6C9005D6602FE024D5
:102E6000FFFDE434FFFC7E007F481253C49005DD73
:102E7000A3E0FEEF8EF0A42416FF9007F37408F091
:102E8000A374FFF0A3740DF0A374F6802DE024FF6B
:102E9000FDE434FFFC7E007F481253C49005DDA39F
:102EA000E0FEEF8EF0A42416FF9007F37408F0A361
:102EB00074FFF0A3740EF0A37402F07B0C7D071274
:102EC0006FDE9005DEE004F070069005DDE004F0B2
:102ED000022E2D9007DBE0FEA3E0FFC394C8EE6452
:102EE000809480500302307DEF94D2EE6480948011
:102EF000400302307D9007F37430F0A374FFF0A319
:102F0000740EF0A3740EF07B117D017F6D126FDEE5
:102F10009007F37430F0A374FFF0A3740DF0A37462
:102F200090F07B117D017F02126FDE9007DBE0FEE7
:102F3000A3E0FF7C007D0A1254197E007FC4125367
:102F4000B274D02FF974133EFA9007F474FFF0A313
:102F5000EAF0A3E9F09007F37438F07B1CE4FD7FFE
:102F600016126FDE9007DBE0FEA3E0FF7C007D0A17
:102F70001254197E007FD81253B274042FF9741BB7
:102F80003EFA9007F474FFF0A3EAF0A3E9F090078B
:102F9000F37420F07B36E4FD7F34126FDE9007DBA4
:102FA000E0FEA3E0FF7C007D0A125419EC7021EDD5
:102FB00014600804701A9005D080039005CEE0FAE2
:102FC000A3E0FB9007E97403F07D047F35126317DB
:102FD000E49005DDF0A3F0900644E0FF9005DDE00D
:102FE000FAA3E0FBC39FEA9400400302307D900700
:102FF000DBE0FEA3E0FF7C007D0A125419EB6D704C
:1030000002EA6C900644602FE024FFFDE434FFFCEC
:103010007E007F481253C49005DDA3E0FEEF8EF0E2
:10302000A42416FF9007F37408F0A374FFF0A374B0
:103030000DF0A374F6802DE024FFFDE434FFFC7E48
:10304000007F481253C49005DDA3E0FEEF8EF0A48C
:103050002416FF9007F37408F0A374FFF0A3740E16
:10306000F0A37402F07B0C7D07126FDE9005DEE0AA
:1030700004F070069005DDE004F0022FD7027AD24A
:105849009007D7E0FCA3E0FDA3E0FEA3E0FF12521E
:10585900D9AB07AA06E4FDFF1271C7900408E0FA64
:10586900A3E0FB9007E97401F07D037F30126EE439
:10587900900422E0FCA3E0FDA3E0FEA3E0FF900773
:10588900E7125489E4FD7F30125E199005CEE0FCE1
:10589900A3E0FDE41252A09007D7E0F8A3E0F9A332
:1058A900E0FAA3E0FB12522250030259459005D0B9
:1058B900E0FCA3E0FDE41252A09007D7E0F8A3E0D2
:1058C900F9A3E0FAA3E0FB1252226002506E9005A0
:1058D900CEE0FCA3E0FDE41252A0A804A905AA06A3
:1058E900AB079007D7E0FCA3E0FDA3E0FEA3E0FF30
:1058F900124F87E4FBFA79C8784212507CC004C081
:1059090005C006C0079005CEE0FEA3E0FFC39005E1
:10591900D1E09FFD9005D0E09EFCE41252A0A804BE
:10592900A905AA06AB07D007D006D005D0041251A5
:10593900851252D99007E8EFF0E4802F9005D0E066
:10594900FCA3E0FDE41252A09007D7E0F8A3E0F928
:10595900A3E0FAA3E0FB125222600B40099007E88A
:105969007464F0E48005E49007E8F0FB7D067F08A5
:10597900126B6C9005CCE0FCA3E0FDEC1252A090F8
:10598900040CE0F8A3E0F9A3E0FAA3E0FB12522229
:10599900607A3000779005CCE0FEA3E0FF7C007DC3
:1059A9000A125419AC06AD07EC1252A090040CE08F
:1059B900F8A3E0F9A3E0FAA3E0FB124F879005C42E
:1059C9001254899005C4E0FCA3E0FDA3E0FEA3E026
:1059D900FF7BCD7ACC794C783F12507C9005C4126C
:1059E90054899005CCE0FEA3E0FF7C007D0A1254A7
:1059F90019AC06AD07EC1252A09005C4E0F8A3E07B
:105A0900F9A3E0FAA3E0FB124F87801C20001F9046
:105A1900040CE0FCA3E0FDA3E0FEA3E0FF7BCD7A4C
:105A2900CC794C783F12507C90040C125489E4FFD5
:105A3900FE7D807C3F90040CE0F8A3E0F9A3E0FA36
:105A4900A3E0FB124F8B1252D99007E8EFF07B01CC
:105A59007D067F41126B6C9005CEE0FEA3E0FFC38B
:105A6900900409E09FFF900408E09EFE7C007D649D
:105A79001253B29005CEE0FCA3E0FDC39005D1E03E
:105A89009DFD9005D0E09CFC1253C4AB07C0039068
:105A99000408E0FFA3E09007E8CFF0A3EFF0900738
:105AA900D7E0FCA3E0FDA3E0FEA3E0FF1252D990EA
:105AB90007EAEEF0A3EFF0D0037D307F0B1260E22E
:105AC9002000139007F37430F0A374FFF0A3740758
:105AD900F0A374C88048900408E0FCA3E0FDE41238
:105AE90052A09007D7E0F8A3E0F9A3E0FAA3E0FBFE
:105AF900124F87E4FBFA79A078401252229007F3FB
:105B09007430500EF0A374FFF0A37406F0A374CCA4
:105B1900800CF0A374FFF0A37405F0A374D0F07B9C
:095B29002AE4FD7F54126FDE2214
:1066DC009007D7E0FCA3E0FDA3E0FEA3E0FF12527D
:1066EC00D9AB07AA06E49007E9F0FDFF126EE4901F
:1066FC000408E0FAA3E0FBE49007E9F07D03FF1245
:10670C006EE49007F3741020000EF0A374FFF0A356
:10671C007424F0A37408800CF0A374FFF0A374230A
:10672C00F0A374E8F07B107D067F04126FDE9007F7
:10673C00F37440F0A374FFF0A37424F0A37428F056
:10674C007B67E4FD7F19126FDE9005DDE4F0A37426
:10675C001AF09005DDE0FEA3E0FFC39480EE9400F8
:10676C005054EF2401FFEF5403703B9005CEE0FE34
:10677C00A3E0FFC39005D1E09FFB9005D0E09EFA0B
:10678C00900408E0FEA3E0FF7C007D3C1253B2AD08
:10679C0003AC021253C4C3743C9FFD9005DDA3E00F
:1067AC00FF7B0112737C9005DEE004F070A4900571
:1067BC00DDE004F0809C200A58E49005DDF0A3F0A5
:1067CC009005DDE0FEA3E0FF24E0F58274053EF5C4
:1067DC0083E0FD74DF2FF58274053EF583EDF090B8
:1067EC0005DEE004F070069005DDE004F09005DDB8
:1067FC00E07004A3E0646470C7D20A9007D7E0FC91
:10680C00A3E0FDA3E0FEA3E0FF1252D9900643EFF4
:10681C00F0E49005DDF0A3F09005DDE0FAA3E0FBD9
:10682C0024DFF58274053AF583E075F03CA4FFAEE5
:10683C00F09005D0E0FCA3E0FD1253C4C3743C9F60
:10684C00FDEB241BFF7B0112737C9005DEE004F052
:10685C0070069005DDE004F0C39005DEE0946590D1
:08686C0005DDE0940040B122BB
:10687400900408E0FCA3E0FDE41252A09007D7E0E6
:10688400F8A3E0F9A3E0FAA3E0FB124F871252D970
:106894009005C2EEF0A3EFF0FDAC06EC1252A0128C
:1068A4007BEAE4FBFA792078411252226018401600
:1068B4009005C2E0FEA3E0FF9005D3E02FF0900521
:1068C400D2E03EF08007E49005D2F0A3F0900402F9
:1068D400E0FEA3E0FF9005C2E0FAA3E0FBC39FFF44
:1068E400EA9E9005BCF0A3EFF09005D4E0FCA3E091
:1068F400FDAF03AE021253B2D3EF94F4EE94014011
:106904000F7E017FF41253C49005C2EEF0A3EFF0A2
:106914009005CAE0FAA3E0FB9005D2E0FEA3E0FFF5
:10692400AD03AC021253B2D3EF94F4EE9401400FD2
:106934007E017FF41253C49005D2EEF0A3EFF090E1
:1069440005C8E0FAA3E0FB9005BCE0FEA3E0FFADC0
:1069540003AC021253B2D3EF94F4EE9401400F7ED1
:10696400017FF41253C49005D2EEF0A3EFF090052A
:10697400D2E0FCA3E0FD9005CAE0FEA3E0FF1253C1
:10698400B2AA06AB079005C2E0FCA3E0FD9005D4D3
:10699400E0FEA3E0FF1253B2EF2BFBEE3AFA9005B0
:1069A400BCE0FCA3E0FD9005C8E0FEA3E0FF1253A9
:1069B400B2EF2BFFEE3AFE9005CCF0A3EFF0D394A8
:1069C400E8EE64809483400A9005CC7403F0A374C9
:1069D400E8F0C39005CCE0648094805004E4F0A314
:1069E400F09005C2E0FFA3E0900402CFF0A3EFF023
:0169F4002280
:107B6900438E805389F0758A66758C7EC28DD28C5E
:037B7900D2A9226C
:107BA000438E0475D78575D6F9438E1043AF0422F2
:107B5400E4FDFCC3ED9FEC9E500A0000000DBD0047
:047B6400010C80EFA1
:017B680022FA
:0E7BCE0075DE2FE4F5BDF5BE7F14FE027B547C
:1075BC00EE6003027650EFB4100040030276509058
:1075CC0075D2F828287302760202760702760C022E
:1075DC00761102761602761B02762002762502764A
:1075EC002A02762F02763402763902763E027643F0
:1075FC0002764802764D75BCC0804975BCC180448A
:10760C0075BCC2803F75BCC3803A75BCC4803575EF
:10761C00BCC5803075BCC6802B75BCC7802675BCBC
:10762C00C8802175BCC9801C75BCCA801775BCCBC1
:10763C00801275BCCC800D75BCCD800875BCCE801D
:10764C000375BCCF7F0A7E00127B54E5BC30E5FB92
:10765C0053BCDFAFBDEFFEADBE7C00E42DFFEC3EB6
:02766C00FE22FC
:0870D5009007E5EEF0A3EFF0D7
:1070DD00FDAC06E41252A09007E7E0F8A3E0F9A397
:1070ED00E0FAA3E0FB12507CC004C005C006C00747
:1070FD009007E5E0FCA3E0FDE41252A0D003D0021E
:10710D00D001D00012507CC004C005C006C007904D
:10711D0007E5E0FCA3E0FDE41252A0D003D002D0BD
:10712D0001D00012507CC004C005C006C0079007F6
:10713D00E5E0FCA3E0FDE41252A09007EBE0F8A31C
:10714D00E0F9A3E0FAA3E0FB12507CC004C005C037
:10715D0006C0079007E5E0FCA3E0FDE41252A0D0C5
:10716D0003D002D001D00012507CD003D002D00148
:10717D00D000124F8BC004C005C006C0079007E5B4
:10718D00E0FCA3E0FDE41252A09007EFE0F8A3E0CD
:10719D00F9A3E0FAA3E0FB12507CD003D002D0019A
:1071AD00D000124F8B9007F3E0F8A3E0F9A3E0FABB
:0971BD00A3E0FB124F8B1252D922
:0171C60022A6
:1041F7000000000000000000002F00000000070082
:10420700070000147F147F1400242A7F2A120062FB
:1042170064081323003649552250000005030000A7
:1042270000001C224100000041221C000014083E2F
:1042370008140008083E0808000000A060000008F5
:104247000808080800006060000000201008040249
:10425700003E5149453E0000427F40000042615107
:104267004946002141454B31001814127F100027A1
:1042770045454539003C4A49493000017109050364
:1042870000364949493600064949291E0000363695
:1042970000000000563600000008142241000014F8
:1042A70014141414000041221408000201510906D5
:1042B70000324959513E007C1211127C007F494956
:1042C7004936003E41414122007F4141221C007F87
:1042D70049494941007F09090901003E4149497A95
:1042E700007F0808087F0000417F4100002040410F
:1042F7003F01007F08142241007F40404040007F7B
:10430700020C027F007F0408107F003E4141413EBE
:10431700007F09090906003E4151215E007F091906
:1043270029460046494949310001017F0101003F03
:104337004040403F001F2040201F003F4038403F83
:1043470000631408146300070870080700615149E7
:10435700454300007F41410000552A552A5500007A
:1043670041417F0000013E4141222060FF60200063
:104377002060FF602000002054545478007F484498
:10438700443800384444442000384444487F0038C7
:104397005454541800087E0901020018A4A4A47CF0
:1043A700007F080404780000447D400000408084BA
:1043B7007D00007F102844000000417F4000007C02
:1043C70004180478007C080404780038444444380E
:1043D70000FC242424180018242418FC007C08045A
:1043E700040800485454542000043F444020003C33
:1043F7004040207C001C2040201C003C4030403CBA
:10440700004428102844001CA0A0A07C0044645449
:104417004C4414141414141400000000000000008D
:104427000000000000000000000000F8000000008D
:10443700000000333000000000100C06100C0600CE
:10444700000000000000000040C07840C078400035
:10445700043F04043F040400007088FC0830000097
:10446700001820FF211E0000F008F000E0180000EF
:1044770000211C031E211E0000F0088870000000A8
:104487001E2123241927211010160E0000000000FA
:104497000000000000000000000000E01804020017
:1044A700000000071820400000020418E000000088
:1044B7000040201807000000404080F08040400086
:1044C7000202010F01020200000000F000000000DC
:1044D7000101011F010101000000000000000000B0
:1044E70080B0700000000000000000000000000025
:1044F70000010101010101010000000000000000AE
:1045070000000000000003030000000080601804A2
:10451700006018060100000000E010080810E00025
:10452700000F102020100F00001010F800000000EE
:104537000020203F20200000007008080888700035
:1045470000302824222130000030088888483000B5
:104557000018202020110E000000C02010F80000D5
:1045670000070424243F240000F80888880808006E
:104577000019212020110E0000E010888818000083
:10458700000F112020110E0000380808C838080055
:104597000000003F000000000070880808887000D5
:1045A700001C222121221C0000E010080810E00056
:1045B7000000312222110F00000000C0C0000000DF
:1045C7000000003030000000000000800000000004
:1045D70000008060000000000000804020100800FC
:1045E70000010204081020004040404040404000C5
:1045F70004040404040404000008102040800000A0
:104607000020100804020100007048080808F000A4
:104617000000003036010000C030C828E810E00074
:104627000718272423140B000000C038E0000000FF
:10463700203C23020227382008F888888870000069
:10464700203F202020110E00C0300808080838003D
:10465700071820202010080008F808080810E000B4
:10466700203F202020100F0008F88888E808100055
:10467700203F20202320180008F88888E808100029
:10468700203F200003000000C03008080838000061
:1046970007182020221E020008F808000008F80862
:1046A700203F210101213F20000808F808080000E9
:1046B7000020203F2020000000000808F80808001C
:1046C700C08080807F00000008F888C02818080094
:1046D700203F20012638200008F8080000000000CD
:1046E700203F20202020300008F8F800F8F80800C4
:1046F700203F003F003F200008F830C00008F808BE
:10470700203F200007183F00E01008080810E000CD
:104717000F10202020100F0008F808080808F000E4
:10472700203F210101010000E01008080810E00007
:104737000F18242438504F0008F88888888870009C
:10474700203F2000030C302000708808080838003C
:104757000038202121221C00180808F80808180032
:104767000000203F2000000008F808000008F808B3
:10477700001F202020201F000878880000C8380864
:10478700000007380E010000F80800F80008F800DC
:10479700033C0700073C0300081868808068180876
:1047A70020302C03032C30200838C800C8380800F4
:1047B7000000203F2000000010080808C838080043
:1047C7002038262120201800000000FE02020200E7
:1047D7000000007F40404000000C30C00000000097
:1047E700000000010638C00000020202FE000000BF
:1047F700004040407F000000000004020202040065
:1048070000000000000000000000000000000000A1
:104817008080808080808080000202040000000089
:104827000000000000000000000080808080000081
:104837000019242222223F2008F80080800000006F
:10484700003F112020110E00000000808080000032
:10485700000E112020201100000000808088F80041
:10486700000E112020103F20000080808080000073
:10487700001F222222221300008080F088888818D7
:104887000020203F202000000000808080808000E2
:10489700006B94949493600008F800808080000077
:1048A700203F210000203F20008098980000000052
:1048B7000020203F20200000000000809898000082
:1048C70000C08080807F000008F8000080808000A2
:1048D700203F24022D302000000808F800000000C7
:1048E7000020203F20200000808080808080800082
:1048F700203F20003F20003F808000808080000014
:10490700203F210000203F200000808080800000A1
:10491700001F202020201F008080008080000000D2
:1049270080FFA12020110E00000000808080800001
:10493700000E112020A0FF808080800080808000F2
:1049470020203F212000010000008080808080001F
:104957000033242424241900008080E08080000094
:104967000000001F202000008080000000808000E1
:10497700001F202020103F20808080000080808042
:1049870000010E30080601008080008000808080D2
:104997000F300C030C300F000080800080808000F7
:1049A7000020312E0E312000808080000080808022
:1049B70080818E70180601000080808080808000D2
:1049C7000021302C2221300000000000807C0202F0
:1049D70000000000003F404000000000FF00000012
:1049E70000000000FF0000000002027C80000000C1
:1049F7000040403F000000001122448811224488F3
:0A4A07000101010102020202088011
:103DEE006400000000000000000000000000000061
:103DFE0000000000000000000000000000000000B5
:103E0E0000000000000000000000000000000000A4
:103E1E000000000000000000000000000000000094
:103E2E000000000000000000000000000000000084
:0841EE0000000000C10EC18DAC
:107AEE00EF4E60157D087C07ED1DAA0470011C4A3F
:097AFE0070F6EF1F70EA1E80E72C
:017B0700225B
:107AB6009007E5EFF07006FD7FA61279E19007E5E5
:0C7AC600E0B40107E4FD7FA71279E12283
:107A08009007E5EFF0700DFD7FC81279E1E4FD7F86
:107A1800A11279E19007E5E0B4010EE4FD7FC01200
:0A7A280079E1E4FD7FA01279E1226C
:020003000022D9
:0F7BB000D2B6D2B5120003C2B6120003C2B5227C
:0A7C0300C2B6D2B5120003D2B622B9
:0F7BBF00D2B6120003D2B5120003C2B502000302
:107A5700E4FEC2B5EF30E704D2B68002C2B6120028
:107A670003D2B5120003C2B5EF25E0FF0EEEB4084E
:017A7700E12D
:017A780022EB
:0A79D7001279E1E4FF1279E17F105C
:1079E100AC07127BB07F78127A57127BBFED60042F
:1079F1007F408002E4FF127A57127BBFAF04127AF4
:077A010057127BBF027C035A
:107A9800AB07ED24B0FFE4FD1279E1EB54F0C454D8
:0E7AA8000F4410FF1279E1EB540FFF0279E159
:107B8F00E4FD7F8D1279E17F141279E17FAF0279E5
:017B9F00E104
:0C7BF700E4FD7F8D1279DC7FAE0279E1A5
:107A7900E4FBEB24B0FFE4FD1279D7E4FA7D01E4DD
:0E7A8900FF1279E10AEAB480F40BEBB408E4D2
:017A970022CC
:086DDC0090080AEFF0A3EDF0AE
:106DE40090080DE0FFC313F9A3F0E4A3F0A3F0EFC0
:106DF400B40809A3E4F0A37406F0802F90080DE012
:106E0400FF131313541FFD7C00EF54077E0060042E
:106E14007F0180027F00EF2DFFEE3CFEE9FD7C0048
:106E24001253B2900811EEF0A3EFF0EB24E0FA90C5
:106E3400080AE0FFA3E0FD127A98E490080FF0A39B
:106E4400F0900811E0FEA3E0FFC3900810E09F90CB
:106E5400080FE09E4003026EE390080EE0FD7C0004
:106E6400A3E0FEA3E0FF1253C4ED4C701590080D8F
:106E7400E06408600D90080AE0FFA3E0FD04F0124E
:106E84007A9890080DE0FBB4081790080FE0FEA371
:106E9400E0FF75F006EAA424F7F582E5F0344180BA
:106EA40019EBB4103A90080FE0FEA3E0FF75F01060
:106EB400EAA4241FF582E5F03444F583E5822FF536
:106EC40082E5833EF583E493FF7D011279E1900826
:0F6ED40010E004F0700690080FE004F0026E4525
:016EE300228C
:077A3200C3EF9E14FD7F0A63
:077A3900900832EFF0A905EF
:107A40007F017E00AD0119ED600C900832E0FD7CF5
:067A5000001253B280EEAB
:017A5600220D
:0E729E00900800EFF0A3EDF0A3EAF0A3EBF0F0
:1072AC00E4900808F0A3F0900805E0B408069008F4
:1072BC00087402F0E4900806F0900804E0FF9008CF
:1072CC0006E0FEC39F4003027371127A32900802EB
:1072DC00E0FCA3E0FDCFCDCFCECCCE1253C47C00CE
:1072EC007D0A1253C4900807EDF0900809E0703C39
:1072FC00900804E014FF900806E0FEC39F502DA3F5
:10730C00E07023900805E0FCC313FF900808E02F01
:10731C008EF0A4FF900800E02FFFA3E0FD90080D75
:10732C00ECF07B2080339008097401F0900805E0A4
:10733C00FEC313FF900808E02FFF900806E0FDEF56
:10734C008DF0A4FF900800E02FFFA3E0FD9008074C
:10735C00E02430FB90080DEEF0126DDC900806E096
:05736C0004F00272C5EF
:0173710022F9
:1078C00090081BEFF0A3EDF0A3EBF0A3EAF0A3E91F
:0178D000F0C7
:1078D100E4900821F090081DE0FBA3E0FAA3E0F991
:1078E100900821E0F582758300125373604090087F
:1078F1001BE0FFA3E0FD900821E0FE04F08E8275FD
:107901008300125373FB900820E090080DF0126D74
:10791100DC900820E0FFB4080990081BE02406F081
:0E79210080B3EFC313FF90081BE02FF080A788
:01792F002235
:107443009007E5EEF0A3EFF0A3ECF0A3EDF0A3EBD0
:01745300F048
:10745400E49007EEF0A3F09007EAE0FF131313544F
:107464001FFEEF540760047F0180027F00EE2F901F
:1074740007EAF0E49007F0F0A3F09007EAE0FF9049
:1074840007F0E0FCA3E0FDC39F7480F8EC648098EF
:1074940050709007E5A3E0FFA3A3E0FEED2EFD12DC
:1074A4007A98E49007F2F0A3F09007E9E0FFC39024
:1074B40007F3E09F7480F89007F2E06480985031FD
:1074C4009007EBE0FBA3E0FAA3E0F9A3E475F00175
:1074D40012546585F082F583125373FF7D0112798E
:1074E400E19007F3E004F070C09007F2E004F0804C
:1074F400B89007F1E004F070819007F0E004F00226
:02750400747E93
:017506002262
:10766E00C2A37FC87E00127AEED2A37FC87E00121C
:10767E007AEEE4FD7FAE1279D77F401279E17F81F9
:10768E001279E17FFF1279E17FA11279E17FC812B1
:10769E0079E17FA61279E17FA81279E17F3F127915
:1076AE00E17FD31279E1E4FF1279E17FD51279E11E
:1076BE007F801279E17FD91279E17FF11279E17F32
:1076CE00DA1279E17F121279E17FDB1279E17F40E4
:1076DE001279E17F201279E17F021279E17F8D121A
:1076EE0079E17F141279E17FA41279E17FA61279F4
:1076FE00E1127A79E4FD7FAF1279E1127A79E4FF33
:0B770E00127AB6E4FF127A08027B8FAB
:0A7372009007ECE0FF9007F0E0FB4D
:0C737C009007FCEBF0AC079007FBEDF075
:1073880020E003E004F0904A10E493FDFF9004002D
:10739800E0FB3395E0FAD3EB9F7480F86A984006D7
:1073A800E4F0A3E004F0904A0FE49375F008A4FF1A
:1073B800900401E0FB3395E0FAD3EB9FE5F064809D
:1073C800F8EA6480984002E4F09007FBE013131396
:1073D800541F8DF0A4AD047C002DFFEC35F0FE7435
:1073E800002FF974003EFA9007FD7401F0A3EAF04B
:1073F800A3E9F09007FBE05407FF7401A807088091
:1074080002C333D8FCFF9007FCE07017A3E0FBA38E
:10741800E475F001125465A9F0FA12535AFEEFF41C
:107428005E80149007FDE0FBA3E475F0011254653B
:0A743800A9F0FA12535A4F1253A0A4
:017442002227
:0B793000900822EBF0A3EAF0A3E9F0BE
:10793B0012535AFF900825E0FBA3E0FAA3E0F912DB
:10794B00535AFE900822E0FBA3E0FAA3E0F9EE12F3
:10795B0053A0900825E0FBA3E0FAA3E0F9EF025354
:01796B00A07B
:105B32009007EDEDF09007ECEFF0F99007EEEBF047
:105B4200E4FA9007F1F0A3F0A312549500000000CC
:105B52009007F712549500000000E9D39B4026906D
:105B620007EEE0FA9007ECE09007EEF09007ECEA1F
:105B7200F09007EFE0FA9007EDE09007EFF0900762
:105B8200EDEAF0E4FA9007EDE0FD9007EFE0FEC3E6
:105B92009D9007F1F09007ECE0FF9007EEE0C39FC5
:105BA2009007F2F0704DEDD39E501C9007EFE0FF8E
:105BB2009007EDE0FDD39F4003025E1812737290CE
:105BC20007EDE004F080E49007EFE0FF9007EDE0DE
:105BD200D39F5003025E189007EDE0FF9007EFE0BD
:105BE200FDD39F4003025E181273729007EFE00428
:105BF200F080E49007F1E0701F9007EEE0FE90075E
:105C0200ECE0FFD39E4003025E18A3E0FD1273771F
:105C12009007ECE004F080E19007F2E0FC1252A55C
:105C2200C004C005C006C0079007F1E0FC1252A5EF
:105C3200D003D002D001D0001251859007F3125444
:105C4200899007EEE0FCE41252A59007F3E0F8A376
:105C5200E0F9A3E0FAA3E0FB12507CC004C005C047
:105C620006C0079007EFE0FCE41252A5D003D00271
:105C7200D001D000124F879007F7125489E4FFFE3B
:105C82007D807CBF9007F3E0F8A3E0F9A3E0FAA3DC
:105C9200E0FB125222600840067F01C00780047FA9
:105CA20000C007E4FFFE7D807C3F9007F3E0F8A38D
:105CB200E0F9A3E0FAA3E0FB12522250047E018035
:105CC200027E00D0E05E60529007EEE0FF9007ECAB
:105CD200E0D39F4003025E18E0FCFFC007E41252CB
:105CE200A59007F3E0F8A3E0F9A3E0FAA3E0FB1222
:105CF200507C9007F7E0F8A3E0F9A3E0FAA3E0FBF9
:105D0200124F8B1252D9AD079007F0E0FBD0071269
:105D1200737C9007ECE004F080AEE4FFFE7D807CB3
:105D2200BF9007F3E0F8A3E0F9A3E0FAA3E0FB12C7
:105D32005222600250067F01C00780047F00C00724
:105D4200E4FFFE7D807C3F9007F3E0F8A3E0F9A337
:105D5200E0FAA3E0FB12522240047E0180027E00A0
:105D6200D0E04E7003025E189007EFE0FF9007ED5F
:105D7200E0D39F504A9007EFE0FF9007EDE0FCD39D
:105D82009F4003025E18E41252A59007F7E0F8A3C1
:105D9200E0F9A3E0FAA3E0FB124F879007F3E0F8E3
:105DA200A3E0F9A3E0FAA3E0FB1251851252D990C5
:105DB20007EDE0FD1273779007EDE004F080B690F6
:105DC20007EFE0FF9007EDE0D39F404A9007EDE038
:105DD200FF9007EFE0FCD39F503CE41252A59007DE
:105DE200F7E0F8A3E0F9A3E0FAA3E0FB124F8790F3
:105DF20007F3E0F8A3E0F9A3E0FAA3E0FB12518570
:105E02001252D99007EFE0FDA3E0FB12737C9007DA
:065E1200EFE004F080B691
:015E18002267
:107AD2009007EA7440F0A37401F0A37400F0A37459
:0C7AE20000F07B80E4FDFCFFFE0274431A
:107B0800904A0FE493FFA3E4938FF0A4FFAEF07DB7
:0A7B1800007B017A0079000254C6D8
:1069F500900828EBF0A3EAF0A3E9F0300D1D90080C
:106A050028E0FBA3E0FAA3E0F9300E0812535AFF81
:106A1500EDF4805F12535A4D026B68200E03026A33
:106A2500CF300F53900828E0FBA3E0FAA3E0F9125A
:106A3500535AFF90082CE0FEC374089EFE74FFA80D
:106A450006088002C333D8FCFEEDF44E5F1253A056
:106A5500900828E0FBA3E0FAA3E0F912535AFF904F
:106A6500082CE0FE74FFA806088002C313D8FCFEBC
:106A7500EDF45E4F026B68900828E0FBA3E0FAA3F3
:106A8500E0F912535AFF90082CE0FEC374089EFEED
:106A950074FFA806088002C313D8FCFEEDF44E5F10
:106AA5001253A0900828E0FBA3E0FAA3E0F91253E3
:106AB5005AFF90082CE0FE74FFA806088002C33335
:106AC500D8FCFEEDF45E4F026B68300F4C90082841
:106AD500E0FBA3E0FAA3E0F912535AFF90082CE07B
:106AE500FEC374089EFE74FFA806088002C333D84F
:106AF500FC4D5F1253A0900828E0FBA3E0FAA3E049
:106B0500F912535AFF90082CE0FE74FFA80608807E
:106B150002C313D8FC5D4F804A900828E0FBA3E030
:106B2500FAA3E0F912535AFF90082CE0FEC374084B
:106B35009EFE74FFA806088002C313D8FC4D5F12A1
:106B450053A0900828E0FBA3E0FAA3E0F912535AFA
:106B5500FF90082CE0FE74FFA806088002C333D816
:076B6500FC5D4F1253A0225A
:0B6CA700900814EDF0900813EFF0FAD5
:106CB200A3E0FE540790081AF0EB24E0900815F0C8
:106CC200EE131313541FFF904A10E493FEEF8EF05D
:106CD200A4FFEA7C002FFFEC35F0FE74002FF9745C
:106CE200003EFA9008177401F0A3EAF0A3E9F0E479
:106CF200900815E075F010A4241FF582E5F03444E5
:106D0200F583E5822CF582E43583F583E493FF90E5
:106D1200081AE0FEEFA806088002C333D8FCFF90F1
:106D22000816F0FDA3E0FBA3E475F001125465A977
:106D3200F0FA90082CEEF0C20F1269F50CECB408D0
:106D4200AF90081AE07003026DDB900814E0FFC3F5
:106D520094304003026DDBEF131313541F75F0647C
:106D6200A4FF900813E07C002FFFEC35F0FE746462
:106D72002FF974003EFA9008177401F0A3EAF0A309
:106D8200E9F0E4900815E075F006A424F7F582E531
:106D9200F03441F583E5822CF582E43583F583E412
:106DA20093FF90081AE0FEC374089EFEEFA806083F
:106DB2008002C313D8FCFF900816F0FDA3E0FBA3EA
:106DC200E475F001125465A9F0FA90082CEEF0D2A5
:096DD2000F1269F50CECB406AADD
:016DDB002295
:097C0D00900400EFF0A3EDF02259
:0875070090082DEFF0A3EDF058
:10750F00E4900831F0900830F090082FF090082E9A
:10751F00E0FFA3E0FEC39F40030275B0127A3290E2
:10752F00082DE0FD7C00CFCDCFCECCCE1253C47C46
:10753F00007D0A1253C4AE05900831E0701B90080D
:10754F002EE014FFA3E0C39F500FEE7006A3E004DC
:10755F00F080459008317401F0900400E0D364800E
:10756F0094DE4007E4F0A3E02408F0900401E0D398
:10757F00648094B04002E4F0900830E0FF90082F50
:10758F00E0C39F75F006A4FF900400E02FFFA3E077
:10759F00FDEE2430FB126CA790082FE004F002756B
:0C75AF001C90082EE0FF900400E02FF07C
:0175BB0022AD
:0F6FDE009007F0EFF09007F2EBF09007F1EDF075
:106FED00FF9007F9E4F0A3EFF09007F3E01313130C
:106FFD00541FFF9007F1E02FFFE433FEC39007FA13
:10700D00E09F9007F9E09E40030270D49007F0E0F6
:10701D00FF9007F7E4F0A3EFF09007F2E0FF900781
:10702D00F0E0F92FFFE433FE9007F7E0FAA3E0FB61
:10703D00C39FEA9E507D9007F1E0FFC39007FAE0F1
:10704D009FFF9007F9E09400FE9007F2E0FD7C00B1
:10705D001253B2E9FDC3EB9DFDEA9CCD2FFFED3E32
:10706D00FE9007F4E0FBA3E0FAA3E0F98F828E8394
:10707D00125373FB904A10E493FF7E009007F9E0E2
:10708D00FCA3E0FD1253B29007F8E02FFF9007F735
:10709D00E03EFE74002FF58274003EF583EBF09018
:1070AD0007F8E004F060030270269007F7E004F0A3
:1070BD000270269007FAE004F06003026FF6900765
:0770CD00F9E004F0026FF688
:0170D4002299
:0E7BDC00E4F5C7F5C5F5C675C3FF75C4FF22F5
:077B2200ECF5C3AF058FC4B1
:107B2900A2AF92D5C2AF75C65A75C6A50000A2D537
:037B390092AF22E6
:1079A500AD07AC0675C78075F52175C501127B223B
:1079B500E5C21253A00DBD00010C740129F9E43A8A
:1079C500FA9007EA74FFF5F012544F45F070DE02A5
:0279D5007BDC59
:107B7C00AD07AC0675C78075F52175C503127B2260
:037B8C00027BDC9D
:10796C00AD07AC0675C78075F52175C502ECF5C37E
:10797C00AF058FC412535AF5C2127B290DBD0001FD
:10798C000C740129F9E43AFA9007EA74FFF5F01245
:09799C00544F45F070D7027BDC6A
:104F8400025345E86480F8E933E83360110460F0C3
:104F9400ED33EC337009E8FCE9FDEAFEEBFF220493
:104FA40060DED3EB9FEA9EE99DE8C2E78CF0C2F78E
:104FB40095F0400CE8CCF8E9CDF9EACEFAEBCFFB5A
:104FC40012531085D0F05804700320D5B3E8047050
:104FD400075002B2D502534F92D5EC0460F7E4CCEB
:104FE400C0E0C398F8603B94186008400DD0E0FB23
:104FF400025327E4FBFAC9FC8028E830E406E4C93C
:10500400FBE4CAFCE830E305E4C9CACBFCE8540776
:105014006010F8C3E913F9EA13FAEB13FBEC13FC81
:10502400D8F130F52FC3E49CFCEF9BFFEE9AFEED24
:1050340099FDD0E0FBEF4E4D4C701222DB0302537E
:105044004CEC2CFCEF33FFEE33FEED33FDED30E79B
:10505400EB025327EF2BFFEE3AFEED39FDD0E0FBD8
:1050640050130BBB000302534FED13FDEE13FEEF81
:0850740013FFEC13FC025327AB
:10507C00EC4D6011E8497017ED33EC3304600DE42E
:10508C00FCFFFEFD22E933E8330470F802534512AD
:10509C00531058046009E4CC2481500628500902AE
:1050AC00534F28400302534CC0E0EB4A7044B98084
:1050BC0006D0E0FB02533BEF4E701CBD8008EBFFAB
:1050CC00EAFEE9FD80EBE98DF0A4FEE5F002516506
:1050DC00E9CDF9EAFEEBFFEF89F0A4FCE5F0CE890F
:1050EC00F0A42EFFE435F0CD89F0A42DFEE435F0CC
:1050FC008067EF4E7005BD80D780C3EF8BF0A4ACFA
:10510C00F0EE8BF0A42CFCE435F0F8EF8AF0A42C34
:10511C00E5F038FCE433CB8DF0A42CFCE5F03BF847
:10512C00EE8AF0A42CFCE5F038F8E433CF89F0A437
:10513C002CFCE5F038CF3400CE89F0A42FFFE5F03D
:10514C003EFEE433C98DF0A42EFEE5F039CD8AF095
:10515C00A42FFFE5F03EFEE43DFD33D0E0FB50070D
:10516C000BBB000F02534FEC2CFCEF33FFEE33FE66
:06517C00ED33FD02532794
:1051820002534FEC5D046005E85904700302534575
:10519200125310580460F6EC4860F2EC7004FDFE05
:1051A200FF22C860DB2481C85009C3986002500600
:1051B20002534C9850CAF582E9294B4A7005AB82DA
:1051C20002533B75F0007C1A7880C3EF9BEE9AED98
:1051D20099400DC3EF9BFFEE9AFEED99FDE842F078
:1051E200DC23ACF0D0E0FFD0E0FED0E0FDAB8220CB
:1051F200E7101BEB60BAEC2CFCEF33FFEE33FEED55
:1052020033FD025327E803F830E705C0F075F000DC
:10521200EF2FFFEE33FEED33FD40B830E7C280AA38
:1052220074F8CC6480CCC86480C8F58204604FC333
:10523200EB9FF5F0EA9E42F0E99D42F0E89C45F0D2
:10524200603C501DE5825FFFE582D313CB5BCBF45C
:105252002B5582FB50280ABA002409B90020088085
:105262001DE5825BFBE582D313CF5FCFF4C3132F1F
:105272005582FF50090EBE00050DBD00010CC3EBA7
:105282009FF5F0EA9E42F0E99D42F0E89C45F0600D
:0952920007CC4820E701B3EC222F
:10529B0075F020800E75F010800575F0087D007E8E
:1052AB00007F003392D530D50312547BEC33401082
:1052BB00EF33FFEE33FEED33FDEC33FCD5F0ED2297
:0E52CB00E5F0247EA2D513CC92E7CDCEFF22D3
:1052D900EDD2E7CD33EC3392D524814006E4FFFECD
:1052E900FDFC22FCE4CFCECDCC24E0501174FF802C
:1052F900EDC3CC13CCCD13CDCE13CECF13CF0470C9
:07530900F030D5DE02547BF9
:0D7BEA00ED33EC3360065004EC6480FC22A7
:10531000E9D2E7C933E833F892D5EDD2E7CD33ECE3
:0753200033FC5002B2D5225C
:10532700EC30E7100FBF000C0EBE00080DBD0004E7
:105337000BEB6014A2D5EB13FCED92E7FD2274FF93
:10534700FCFDFEFF22E480F8A2D574FF13FC7D80EC
:03535700E480EF00
:030000000277BBC9
:0C77BB00787FE4F6D8FD75812102780289
:10535A00BB010689828A83E0225002E722BBFE0251
:09536A00E32289828A83E4932284
:10537300BB010CE58229F582E5833AF583E02250EF
:1053830006E92582F8E622BBFE06E92582F8E22239
:0D539300E58229F582E5833AF583E4932253
:1053A000BB010689828A83F0225002F722BBFE01EC
:0253B000F322E6
:1053B200EF8DF0A4A8F0CF8CF0A428CE8DF0A42E0F
:0253C200FE22C9
:1053C400BC000BBE0029EF8DF084FFADF022E4CCCD
:1053D400F875F008EF2FFFEE33FEEC33FCEE9DEC96
:1053E400984005FCEE9DFE0FD5F0E9E4CEFD22EDDC
:1053F400F8F5F0EE8420D21CFEADF075F008EF2F26
:10540400FFED33FD4007985006D5F0F222C398FD16
:055414000FD5F0EA22B3
:10541900C2D5EC30E709B2D5E4C39DFDE49CFCEEAE
:1054290030E715B2D5E4C39FFFE49EFE1253C4C30F
:10543900E49DFDE49CFC80031253C430D507C3E40A
:065449009FFFE49EFE221D
:10544F00C5F0F8A3E028F0C5F0F8E58215827002E8
:06545F001583E038F02285
:10546500A3F8E0C5F025F0F0E582158270021583FA
:06547500E0C838F0E82257
:0E547B00C3E49FFFE49EFEE49DFDE49CFC2242
:0C548900ECF0A3EDF0A3EEF0A3EFF02296
:10549500A8828583F0D083D0821254AC1254AC120A
:1054A50054AC1254ACE473E493A3C583C5F0C5832F
:1054B500C8C582C8F0A3C583C5F0C583C8C582C861
:0154C50022C4
:1054C600EF4E6012EF60010EEDBB010B89828A83FD
:1054D600F0A3DFFCDEFA2289F05007F709DFFCA90A
:0C54E600F022BBFEFCF309DFFCA9F02261
:1077C700027B3CE493A3F8E493A34003F68001F221
:1077D70008DFF48029E493A3F85407240CC8C333C3
:1077E700C4540F4420C8834004F456800146F6DF92
:1077F700E4800B010204081020408090398DE47E5C
:10780700019360BCA3FF543F30E509541FFEE49386
:10781700A360010ECF54C025E060A840B8E493A34D
:10782700FAE493A3F8E493A3C8C582C8CAC583CA78
:10783700F0A3C8C582C8CAC583CADFE9DEE780BE30
:0141F60000C8
:00000001FF
